:100000000C9454030C9471030C9437200C947103DA
:100010000C9471030C9471030C9471030C94710390
:100020000C9471030C94B2350C9471030C9471030D
:100030000C9471030C9471030C9471030C94710370
:100040000C9471030C9471030C9471030C94710360
:100050000C9471030C94F6410C9471030C94E741D9
:100060000C9471030C9471030C9471030C94710340
:100070000C9471030C9471030C9471030C94710330
:100080000C9471030C9471030C9471030C94710320
:100090000C9471033A3784373F386438D838F938CC
:1000A0002039233932394B3F4B3F4B3F4B3F4B3F7E
:1000B0004B3F4B3F4B3F4B3F4B3F4B3F4B3F4B3FF0
:1000C0004B3F4B3F4B3F4B3F4B3F4B3F4B3F4B3FE0
:1000D0004B3FBD3941395A39DB39EB394B3F4B3F47
:1000E0005F3BA13BDD3B1C3C4B3F4B3F4B3F4B3F02
:1000F0004B3F4B3F4B3F4B3F4B3F4B3F4B3F4B3FB0
:100100004B3F4B3F4B3F4B3F4B3F4B3F4B3F4B3F9F
:100110004B3F1A3A5F3A553C6E3C9E3CAB3C4B3FE2
:100120004B3F4B3F4B3F4B3F4B3F4B3F4B3F4B3F7F
:100130004B3F8F3AE73AB73C303DAC3DEE3D8D3E0C
:100140009C3E653E793EAB3EBD3ED03E4B3FE13EE0
:10015000CC3AF43A1C3B153F303F2F3E4A3ECE038B
:10016000C103B303A30390037A0361034703290385
:100170000803E602C2029E0276024F022802030230
:100180006C01B80196017501560139011F01060184
:10019000EF00DA00B5008200A500960000004341A0
:1001A0004E20310000000000000000000043414EDE
:1001B00020320000000000000000000043414E20FB
:1001C000330000000000000000000043414E2034D6
:1001D0000000000000000000000043414E203500F8
:1001E00000000000000000000043414E20360000E7
:1001F000000000000000000043414E2037000000D6
:100200000000000000000043414E203800000000C4
:1002100000000000000043414E20390000000000B3
:10022000000000000043414E20313000000000007B
:100230000000000043414E2031310000000000006A
:1002400000000043414E2031320000000000000059
:10025000000043414E203133000000000000000048
:100260000043414E20313400000000000000000037
:1002700043414E20313500000000000000000043E3
:10028000414E2031360000000000000000004341D4
:100290004E20313700000000000000000043414EB6
:1002A00020313800000000000000000043414E20D3
:1002B000313900000000000000000043414E2032B0
:1002C0003000000000000000000043414E203231A9
:1002D000000000000000000000466C6173682031DF
:1002E0000000000000000000466C617368203200CE
:1002F00000000000000000466C61736820330000BD
:10030000000000000000466C6173682034000000AB
:100310000000000000466C6173682035000000009A
:1003200000000000535749544348203100000000AA
:100330000000005357495443482032000000000099
:100340000000535749544348203300000000000088
:100350000053574954434820340000000000000077
:100360005357495443482035000000000000005313
:1003700057495443482036000000000000005357FE
:1003800049544348203700000000000000535749FB
:1003900054434820380000000000000053574954DF
:1003A00043482039000000000000005357495443DF
:1003B00048203130000000000000535749544348A2
:1003C0002031310000000000004348414E4E454CB2
:1003D00020310000000000004348414E4E454C20B3
:1003E000320000000000004348414E4E454C20338F
:1003F0000000000000004348414E4E454C203400B0
:1004000000000000004348414E4E454C203500009E
:10041000000000004348414E4E454C20360000008D
:100420000000004348414E4E454C2037000000007C
:1004300000004348414E4E454C203800000000006B
:10044000004348414E4E454C20390000000000005A
:100450004348414E4E454C203130000000000043DF
:1004600048414E4E454C20313100000000004348C9
:10047000414E4E454C2031320000000000434841BF
:100480004E4E454C20313300000000004348414EA1
:100490004E454C20313400000000004348414E4E90
:1004A000454C20313500000000004348414E4E4588
:1004B0004C20313600000000004348414E4E454C70
:1004C00020313700000000004348414E4E454C208B
:1004D000313800000000004348414E4E454C203169
:1004E0003900000000004348414E4E454C20323058
:1004F00000000000004348414E4E454C2032310080
:10050000000000004348414E4E454C20323200006E
:100510000000004348414E4E454C2032330000005D
:1005200000004348414E4E454C203234000000004C
:10053000004348414E4E454C20323500000000003B
:100540004348414E4E454C203236000000000043E7
:1005500048414E4E454C20323700000000004348D1
:10056000414E4E454C2032380000000000434841C7
:100570004E4E454C20323900000000004348414EA9
:100580004E454C20333000000000004348414E4EA1
:10059000454C20333100000000004348414E4E4599
:1005A0004C20333200000000004348414E4E454C81
:1005B00020333300000000004348414E4E454C209C
:1005C000333400000000005649525455414C20314C
:1005D0000000000000005649525455414C203200A2
:1005E00000000000005649525455414C2033000091
:1005F000000000005649525455414C203400000080
:100600000000005649525455414C2035000000006E
:1006100000005649525455414C203600000000005D
:10062000005649525455414C20370000000000004C
:100630005649525455414C203800000000000056E5
:1006400049525455414C20390000000000005649E1
:10065000525455414C2031300000000000564952A0
:100660005455414C2031310000000000564952548D
:1006700055414C203132000000000056495254557B
:10068000414C20313300000000005649525455417E
:100690004C20313400000000005649525455414C62
:1006A000203135000000000011241FBECFEFD0E143
:1006B000DEBFCDBF11E0A0E0B1E0E2E9F5EA00E085
:1006C0000BBF02C007900D92AA37B107D9F71EE001
:1006D000AAE7B1E001C01D92AF31B107E1F70C9478
:1006E00027280C940000282F277099279695879526
:1006F000969587959695879533272330310529F16F
:10070000243031054CF421303105B9F02230310567
:10071000C4F4232B71F02CC025303105F1F02530C5
:100720003105BCF026303105E1F027303105E9F024
:100730001FC0A098A198A2981BC0A09AA198A298A7
:1007400017C0A098A19AA29813C0A09AA19AA298A3
:100750000FC0A098A198A29A0BC0A09AA198A29AA3
:1007600007C0A098A19AA29A03C0A09AA19AA29A9F
:10077000806280937C0080917A00806480937A000C
:1007800080917A0084FFFCCF80917A008061809311
:100790007A0020917800809179009927880F991F1D
:1007A000880F991F2295269526952370820F911DFB
:1007B0000895282F27709927969587959695879560
:1007C0009695879533272330310529F1243031055B
:1007D0004CF421303105B9F022303105C4F4232B1B
:1007E00071F02CC025303105F1F025303105BCF019
:1007F00026303105E1F027303105E9F01FC0A0981F
:10080000A198A2981BC0A09AA198A29817C0A098DE
:10081000A19AA29813C0A09AA19AA2980FC0A098DA
:10082000A198A29A0BC0A09AA198A29A07C0A098DA
:10083000A19AA29A03C0A09AA19AA29A80628093D8
:100840007C0080917A00806480937A0080917A00A5
:1008500084FFFCCF80917A00806180937A00809140
:1008600079009927089540E050E0FC010296259117
:1008700034916217730760F44B5F5F4FFC0102967F
:10088000259134916217730718F446395105A4F382
:10089000CA010895FC01809100018130B1F41092E9
:1008A0000001F0938301E0938201F0938101E093D2
:1008B0008001F0937F01E0937E01F0937D01E0934E
:1008C0007C01F0937B01E0937A016091800170914B
:1008D0008101709383016093820140917E01509168
:1008E0007F01509381014093800120917C013091E0
:1008F0007D0130937F0120937E0180917A01909158
:100900007B0190937D0180937C01F0937B01E093C8
:100910007A01E80FF91FE20FF31FE40FF51FCF0173
:10092000860F971F65E070E00E941052CB0108957A
:1009300080E10E9473030E944A04BC018EE591E0AD
:100940000E9433049927089583E10E94D9039FE40C
:10095000899FC0011124880F892F881F990B9195B9
:10096000A82F809101018130C1F4109201018A2FDA
:10097000992790938D0180938C0190938B018093A4
:100980008A019093890180938801909387018093D5
:1009900086019093850180938401E0918A01F09112
:1009A0008B01F0938D01E0938C016091880170912F
:1009B000890170938B0160938A0140918601509167
:1009C00087015093890140938801209184013091DF
:1009D000850130938701209386018A2F9927909370
:1009E000850180938401820F931F840F951F860FCA
:1009F000971F8E0F9F1F65E070E00E941052862F98
:100A00009927089580E280937C0087E880937A009C
:100A1000989A999A9A9AA098A198A298089590E085
:100A2000892F8295807F8093ED001092EE001092C6
:100A3000EF001092F0001092F1001092F20010926C
:100A4000F3001092F4001092F5001092F60010924C
:100A5000F70080E01092FA008F5F8830D8F39F5F34
:100A60009F30F0F208953091ED0090E020EC892F56
:100A70008295807F8093ED008091EF00822329F49E
:100A80003093ED00892F992708959F5F9F3078F369
:100A90003093ED008FEF90E008958091EE0086FF97
:100AA00003C080E090E008958091EE0085FF03C0D0
:100AB00081E090E008958091EF00807C19F48FEF41
:100AC00090E0089582E090E00895BC0140E08091BC
:100AD000EF0099278F709070892B89F0FB01E40F4C
:100AE000F11D8091FA0080834F5F242F332780917E
:100AF000EF0099278F709070281739077CF30895BD
:100B000089EC9CE00E9478276FE67DE080E00E94FF
:100B1000B52767E27DE081E00E94B52761EE7CE0C9
:100B200082E00E94B52781E080938E018091C90CFC
:100B3000813061F48091CA0C9091CB0C6AE070E036
:100B40000E9410527093C80C6093C70C8091700D76
:100B5000813061F48091710D9091720D6AE070E0C6
:100B60000E9410527093C40C6093C30C8091280DA6
:100B7000813061F48091290D90912A0D6AE070E036
:100B80000E9410527093C60C6093C50C8091E20CC9
:100B9000813061F48091E30C9091E40C6AE070E0A4
:100BA0000E94105270936E0D60936D0D0895CF9357
:100BB000DF93CDB7DEB7CE55D0400FB6F894DEBF89
:100BC0000FBECDBF19828CE0888F84E690E09B83B6
:100BD0008A831D821C821E821F82188619861A86AD
:100BE0001B8689819E01245F3F4FF901E80FF11DAB
:100BF00010828F5F8C30C8F3CE0101960E94682767
:100C0000A895198E1A8E84E690E09C8F8B8F1E8E8D
:100C10001D8E898D9E012F5F3F4FF901E80FF11D59
:100C2000168E8F5F8232C8F3CE0149960E948827C4
:100C3000A89581E0898F1A8E84E690E09C8F8B8F37
:100C40001E8E1D8E8A8D9E012F5F3F4FF901E80F8A
:100C5000F11D168E8F5F8232C8F3CE0149960E9435
:100C60008827A89582E0898F1A8E84E690E09C8F71
:100C70008B8F1E8E1D8E8A8D9E012F5F3F4FF90137
:100C8000E80FF11D168E8F5F8034C8F3CE014996B0
:100C90000E948827C25ADF4F0FB6F894DEBF0FBEFE
:100CA000CDBFDF91CF910895FF920F931F93CF9304
:100CB000DF93CDB7DEB765970FB6F894DEBF0FBEF2
:100CC000CDBF8091C70C9091C80C009709F479C0F2
:100CD00001979093C80C8093C70C892B09F071C0C1
:100CE0008091CA0C9091CB0C6AE070E00E94105287
:100CF0007093C80C6093C70C8091CC0C9091CD0C74
:100D0000AA27BB2789839A83AB83BC8388E08D8322
:100D100080918E018E838091CE0C0E94B11E96959B
:100D20008795969587958F838091CF0C0E94B11EF1
:100D3000969587959695879588878091D00C0E9487
:100D4000B11E969587959695879589878091D10C48
:100D50000E94B11E96958795969587958A87809172
:100D6000D20C0E94B11E96958795969587958B8794
:100D70008091D30C0E94B11E969587959695879584
:100D80008C8720918E0189EC9CE0FC01E20FF11D23
:100D900082850E94B11E96958795969587958D8739
:100DA00080918E01982F9F5F90938E018091E00C2F
:100DB000891718F481E080938E01CE0101960E947C
:100DC000E2328091C30C9091C40C009709F48DC05D
:100DD00001979093C40C8093C30C892B09F085C0B4
:100DE000CE010E960E941B1E8091710D9091720D86
:100DF0006AE070E00E9410527093C40C6093C30CC0
:100E00008091730D9091740DAA27BB2789839A83D3
:100E1000AB83BC8388E08D83FF2400E81F2D812FE6
:100E20009927FC01E159F24F86810E94D51D81115D
:100E3000F02A06951F5F183090F3FE82FF2400E829
:100E40001F2D812F9927FC01E159F24F86850E94C1
:100E5000D51D8111F02A06951F5F183090F3FF828F
:100E6000FF2400E81F2D812F9927FC01E159F24F43
:100E700086890E94D51D8111F02A06951F5F1830C2
:100E800090F3F886FF2400E81F2D812F9927FC019D
:100E9000E159F24F868D0E94D51D8111F02A0695E9
:100EA0001F5F183090F3F986FF248091950D0E9402
:100EB000D51D882321F00F2EF0E8FF2EF02D809114
:100EC000960D0E94D51D882311F080E4F82AFA8639
:100ED0008E859F856AE070E00E9410526B871C86A9
:100EE0001D86CE0101960E94E2328091C50C909140
:100EF000C60C009709F489C001979093C60C8093A3
:100F0000C50C892B09F081C08091290D90912A0D83
:100F10006AE070E00E9410527093C60C6093C50C9A
:100F200080912B0D90912C0DAA27BB2789839A8342
:100F3000AB83BC8388E08D83FF2400E81F2D812FC5
:100F40009927FC01E95DF24F86810E94FB1D81110A
:100F5000F02A06951F5F183090F3FE82FF2400E808
:100F60001F2D812F9927FC01E95DF24F86850E9494
:100F7000FB1D8111F02A06951F5F183090F3FF8248
:100F8000FF2400E81F2D812F9927FC01E95DF24F16
:100F900086890E94FB1D8111F02A06951F5F18307B
:100FA00090F3F886FF2400E81F2D812F9927FC017C
:100FB000E95DF24F868D0E94FB1D8111F02A069596
:100FC0001F5F183090F3F986FF2480914D0D0E9429
:100FD000FB1D882321F00F2EF0E8FF2EF02D8091CD
:100FE0004E0D0E94FB1D882311F080E4F82AFA863A
:100FF0008E859F856AE070E00E9410526B871C8688
:101000001D86CE0101960E94E23280916D0D909175
:101010006E0D009709F4B4C0019790936E0D809304
:101020006D0D892B09F0ACC08091E30C9091E40C1C
:101030006AE070E00E94105270936E0D60936D0D27
:101040008091E50C9091E60CAA27BB2789839A83AF
:10105000AB83BC8388E08D83FF2400E81F2D812FA4
:101060009927FC01EF51F34F86810E94D51D811114
:10107000F02A06951F5F183090F3FE82FF2400E8E7
:101080001F2D812F9927FC01EF51F34F86850E9478
:10109000D51D8111F02A06951F5F183090F3FF824D
:1010A000FF2400E81F2D812F9927FC01EF51F34FFA
:1010B00086890E94D51D8111F02A06951F5F183080
:1010C00090F3F886FF2400E81F2D812F9927FC015B
:1010D000EF51F34F868D0E94D51D8111F02A0695A0
:1010E0001F5F183090F3F986FF2400E81F2D812F31
:1010F0009927FC01EF51F34F86A10E94FB1D81113E
:10110000F02A06951F5F183090F3FA86FF2400E856
:101110001F2D812F9927FC01EF51F34F86A50E94C7
:10112000FB1D8111F02A06951F5F183090F3FB8696
:10113000FF2400E81F2D812F9927FC01EF51F34F69
:1011400086A90E94FB1D8111F02A06951F5F1830A9
:1011500090F3FC86FF2400E81F2D812F9927FC01C6
:10116000E15EF24F80810E94FB1D8111F02A0695FD
:101170001F5F183090F3FD86CE0101960E94E23287
:1011800065960FB6F894DEBF0FBECDBFDF91CF914D
:101190001F910F91FF9008958F929F92BF92CF92CF
:1011A000DF92EF92FF920F931F93CF93DF93CDB710
:1011B000DEB7EC970FB6F894DEBF0FBECDBFBB24F1
:1011C0000F2EF3E18F2E9924F02DBE016F5F7F4F1C
:1011D0008B2D0E949E258B2D9927889D9001899D9E
:1011E000300D989D300D11240F2EFFE8CF2EF1E029
:1011F000DF2EF02DC20ED31E8981F60180838A81F5
:101200009B81928381838C819D81948383832E81B2
:101210003F813683258388859985908787839A8542
:1012200091878B8582878C8583878D8584878E8542
:1012300085878F8586878F8D878788A1808B89A1F9
:10124000818B8AA1828B933090F5C901AA2797FDE3
:10125000A095BA2FBC01CD010E94354FDC01CB0116
:1012600028A539A54AA55BA5BC01CD010E944F4E1A
:101270007B018C018CA5992787FD9095A92FB92F0B
:10128000BC01CD010E94354FDC01CB019C01AD01B9
:10129000C801B7010E941A4EDC01CB01BC01CD018F
:1012A0000E949B4CDC01CB01F601968385838B2D3C
:1012B0009927889D9001899D300D989D300D1124AE
:1012C0000F2EFFE8CF2EF1E0DF2EF02DC20ED31E41
:1012D000F6018285833098F588859985AA2797FD40
:1012E000A095BA2FBC01CD010E94354FDC01CB0186
:1012F00028A539A54AA55BA5BC01CD010E944F4E8A
:101300007B018C018CA5992787FD9095A92FB92F7A
:10131000BC01CD010E94354FDC01CB019C01AD0128
:10132000C801B7010E941A4EDC01CB01BC01CD01FE
:101330000E949B4CDC01CB01F601908787838B2DAB
:101340009927FC01E25EFC4F1082FC01EE5BFC4F32
:101350001082B394F4E1FB1508F037CFFE01BD967F
:10136000A0E9B7E080E190E021E08030920719F435
:101370000E94B35203C0182E0E94B3528DA58093D1
:1013800040038EA58093410381E080933403109243
:101390003303EC960FB6F894DEBF0FBECDBFDF91DE
:1013A000CF911F910F91FF90EF90DF90CF90BF9062
:1013B0009F908F9008951F93CF93DF93CDB7DEB7A3
:1013C000EC970FB6F894DEBF0FBECDBF10E0A89526
:1013D00019821B821A821D821C821F821E8219861C
:1013E00018861A861B861C8681E08D871E868F874D
:1013F0001F8E18A219A21AA280E090E0A0E8BFE315
:1014000088A799A7AAA7BBA71CA685E0FE01B3964B
:1014100011928A95E9F78FE0FE017096DF01282F7F
:101420001D922A95E9F7189FC001112482569E4FFC
:10143000BC01CF010E94C051BE016F5F7F4F812F61
:101440000E9466251F5F153110F2FE01BD9680E1F6
:10145000DF011D928A95E9F7A0E9B7E080E190E00D
:1014600021E08030920719F40E94C45203C0182E64
:101470000E94C452EC960FB6F894DEBF0FBECDBFEB
:10148000DF91CF911F9108958093330308950F93B7
:10149000CF93DF93CDB7DEB721970FB6F894DEBFB9
:1014A0000FBECDBF89838150853170F000E021E00F
:1014B000AE014F5F5F4F61EE70E082E091E00E940D
:1014C000692180E090E007C089819927FC01E35EF3
:1014D000FC4F8081992721960FB6F894DEBF0FBE8E
:1014E000CDBFDF91CF910F91089580914003882364
:1014F00079F0809141030E94B034882349F42EE1B1
:1015000033E0F901E80FF11D10828F5F8531C8F3D8
:1015100080E022E433E04EE153E0E82FFF27DF01D3
:10152000A20FB31F9C91992339F091509C9399235A
:1015300019F4E40FF51F90838F5F853170F30895E0
:10154000809133038823A1F080913403882381F4B0
:1015500084E393E0AC014C5F5F4F6091370380916F
:101560003503909136030E94913F81E080933403CC
:101570000895AF92BF92DF92EF92FF920F931F9365
:10158000CF93DF938C01EE24FF24DD248091400370
:10159000882339F0809141030E94B034882309F4F4
:1015A000B2C160E00F2EFEE1AF2EF3E0BF2EF02DB2
:1015B00071E083E1689FC0011124EC01C157DE4F47
:1015C00089819A81AA2797FDA095BA2FF8012081D9
:1015D00031814281538182179307A407B50759F0DF
:1015E0008B819C81AA2797FDA095BA2F821793071C
:1015F000A407B50739F482E493E0FC01E60FF11D7E
:101600008FE080838F85882349F08889F801E80F6F
:10161000F11D99898581981709F050C129813A8176
:101620002115310509F44AC1442737FD4095542F4F
:10163000F80180819181A281B381281739074A0777
:101640005B0709F094C0DD24D3942D2D8B8588236E
:1016500071F0E80FF11D84819927F82EEE248C8516
:10166000F801E80FF11D8481E80EF11C0BC08C8598
:10167000882339F0F801E80FF11D8481E82EFF245A
:1016800001C020E0222309F472C0898599278230A5
:101690009105B9F1833091052CF4009779F0019709
:1016A000C1F065C08430910509F44DC084309105C6
:1016B0000CF43EC0059709F451C059C08D819E813C
:1016C0008E159F0509F053C0F501E60FF11D7083DB
:1016D0004EC02A89213059F48D819E818E159F0537
:1016E0000CF045C0F501E60FF11D208340C08D814F
:1016F0009E818E159F05D8F5F501E60FF11D7083CB
:1017000036C02A89213051F48D819E81E816F90670
:1017100074F5F501E60FF11D208329C08D819E81AE
:10172000E816F90620F5F501E60FF11D70831FC0DC
:101730008D819E818E219F21892BC9F0F501E60FB5
:10174000F11D708314C08D819E818E219F21892B74
:1017500071F4F501E60FF11D708309C08D819E8142
:101760008E159F0521F0F501E60FF11D70838B8129
:101770009C819C01442737FD4095542FF8018081BE
:101780009181A281B381281739074A075B0709F0C5
:1017900095C0DD24D3942D2D8D85882379F0E80F15
:1017A000F11D8481E82EFF24FE2CEE248E85F801A5
:1017B000E80FF11D8481E80EF11C0BC08E85882393
:1017C00039F0F801E80FF11D8481E82EFF2401C0F3
:1017D00020E0222309F472C08A859927823091057E
:1017E000B9F1833091052CF4009779F00197C1F09D
:1017F00065C08430910509F44DC0843091050CF426
:101800003EC0059709F451C059C08F8198858E1547
:101810009F0509F053C0F501E60FF11D10824EC07F
:101820002A89213059F48F8198858E159F050CF0F7
:1018300045C0F501E60FF11D208340C08F819885DA
:101840008E159F05D8F5F501E60FF11D108236C003
:101850002A89213051F48F819885E816F90674F5AC
:10186000F501E60FF11D208329C08F819885E816C8
:10187000F90620F5F501E60FF11D10821FC08F81DA
:1018800098858E219F21892BC9F0F501E60FF11D66
:10189000108214C08F8198858E219F21892B71F42D
:1018A000F501E60FF11D108209C08F8198858E1514
:1018B0009F0521F0F501E60FF11D10826F5F653184
:1018C00008F477CE809133038823E9F0DD20D9F046
:1018D000809134038130B9F410923403F80180818F
:1018E00091819093360380933503848180933703ED
:1018F000992798012B5F3F4FAC01B90184E393E036
:1019000004960E94C751DF91CF911F910F91FF90D4
:10191000EF90DF90BF90AF90089582E08093E20057
:1019200084E08093E30083E18093E4000E940F054C
:101930008091D80082608093D8000895CF93DF9380
:10194000EC018981833089F48985882309F403C1F6
:1019500088818295807F8093ED008091EF008F7366
:101960008093EF0018821986F6C00E943305982FE5
:1019700081E089879F3F09F4EBC09883892F829586
:10198000807F8093ED001092EE001092EF00109295
:10199000F7001092F6001092F5001092F4001092E9
:1019A000F000898199278130910509F46BC082305C
:1019B00091051CF4892B29F0C9C0029709F4BBC01A
:1019C000C5C08A8581FF30C08D81982F990F990FEE
:1019D000990F8C81829586958770890F8093F3008B
:1019E0008C81982F990F990F990F8B8182958695ED
:1019F0008770890F8093F2008B81982F990F990F30
:101A0000990F8A81829586958770890F8093F1005E
:101A10008A81880F880F880F8093F0008091EF00F3
:101A200080618093EF0012C08B81982F9295990F5F
:101A3000907E8A81869586958695890F8093F3009E
:101A40008A818295880F807E8093F20020E08E81CB
:101A5000181660F48F819885FC01E20FF11D8081DA
:101A60008093FA002F5F8E812817A0F39091EF00EA
:101A70008E81892B8093EF008091EF0080648093AA
:101A8000EF0069C08A8581FF35C08D81982F990F3D
:101A9000990F990F8C81829586958770890F809315
:101AA000F3008C81982F990F990F990F8B81829554
:101AB00086958770890F8093F2008B81982F990FFC
:101AC000990F990F8A81829586958770890F8093E7
:101AD000F1008A81880F880F880F8093F000809131
:101AE000EF0080618093EF008091F000846080932C
:101AF000F00015C08B81982F9295990F907E8A8166
:101B0000869586958695890F8093F3008A818295C4
:101B1000880F807E8093F20084E08093F0009091A3
:101B2000EF008E81892B8093EF008091EF0080641D
:101B30008093EF0010C08091EF008F738093EF00CF
:101B40008091EF0080688093EF0005C0198603C084
:101B50008FEF90E002C080E090E0DF91CF91089598
:101B6000CF93DF93EC018985882319F482E090E01C
:101B700082C088818295807F8093ED000E944D0510
:101B8000813009F06CC019868091EF008F708E83D0
:101B90008F8198850E9465058091F0009927847057
:101BA00090709595879595958795982F91708A85D2
:101BB000282F2E7F292B2A878091EF0084FF31C0A8
:101BC000822F82608A878091F3008695869586951C
:101BD0008D838091F200982F969596959695809199
:101BE000F3008295880F807E890F8C838091F100AD
:101BF000982F9695969596958091F2008295880FEC
:101C0000807E890F8B838091F000982F9695969512
:101C100096958091F1008295880F807E890F8A8346
:101C200016C08A858D7F8A878091F300829586957C
:101C300087708B838091F200982F9295969597707C
:101C40008091F300880F880F880F890F8A83809115
:101C5000EF008F738093EF0080E090E00CC088234A
:101C600049F489878091EF008F738093EF0080E0C3
:101C700090E001C09927DF91CF9108958EEC98E014
:101C80000E94C11F0E94E40E08951F93CF93DF931B
:101C90000E9413160E94A6150E944A1710E087E2C0
:101CA000189FC0011124EC01C25ADC4F8C899D8918
:101CB000009719F001979D8B8C8B8D859E850097E1
:101CC00061F001979E878D8799859F3F31F085E070
:101CD000989FC00111249B878A872A853B852115FF
:101CE000310561F089858F3F49F0C90101979B87D4
:101CF0008A87892B19F48F8580628F878B8D9C8DC5
:101D0000009779F001979C8F8B8F892B51F48F85E9
:101D100086FD04C0812F8F5F0E9447248F858064D9
:101D20008F878F81882311F081508F831F5F12323C
:101D300008F4B5CFDF91CF911F9108950E94D1296A
:101D40009091C5088091D5089817E0F420E045ED02
:101D500058E067E270E0FA01E20FF11D8281823201
:101D600068F49927869FF001879FF00D969FF00DEC
:101D70001124EE59FC4F8081816080832F5F2C30CD
:101D800050F308959091C5088091D6088917D8F42A
:101D900020E045ED58E067E270E0FA01E20FF11D46
:101DA0008281823268F49927869FF001879FF00D27
:101DB000969FF00D1124EE59FC4F80818E7F808319
:101DC0002F5F2C3050F30895CF92DF92EF92FF9265
:101DD0000F931F93CF93DF9380915803882309F0CB
:101DE000FDC0F82E0F2EFAE0EF2EF02D8DE0F89EBC
:101DF000C0011124EC01C450D74F00E08A818F3F0D
:101E000011F401E01DC09A81892F805C843128F48F
:101E1000892F0E94B034082F13C09A81892F8150D6
:101E20008F3028F4892F0E94470A082F09C09A8111
:101E3000892F86518A3020F4892F0E942C45082F43
:101E40008981992781309105C9F1823091051CF46F
:101E5000892B29F0BEC0029709F4B8C0BAC001307E
:101E600009F0B7C08F818E9DC00111249C838B83A4
:101E700088858E9DC00111249E838D838881846016
:101E8000888310E027E230E0FE01E10FF11D81853B
:101E90008F3F71F09927829FA001839F500D929FE1
:101EA000500D1124FA01EE59FC4F8081846080832B
:101EB0001F5F143048F381E089838BC08B819C8144
:101EC000009709F486C001979C838B83892B49F581
:101ED0008F818E9DC00111249C838B83888182FF1A
:101EE00010C08B7F888310E0FE01E10FF11D81851A
:101EF0008F3F19F060E00E94F70F1F5F1430A0F3CE
:101F000010C088818460888310E0FE01E10FF11D1C
:101F100081858F3F19F061E00E94F70F1F5F143039
:101F2000A0F38881282F227081FD28C08D819E8199
:101F3000009709F44EC001979E838D83892B09F089
:101F400048C082E08983122F27E230E0FE01E10FD2
:101F5000F11D81858F3F71F09927829FA001839F9A
:101F6000500D929F500D1124FA01EE59FC4F8081C3
:101F70008B7F80831F5F143048F32BC0002349F50B
:101F8000102F0F2EF7E2CF2EDD24F02DFE01E10FF2
:101F9000F11D21852F3F99F0822F99278C9DA0015B
:101FA0008D9D500D9C9D500D1124FA01EE59FC4F52
:101FB00080818B7F808361E0822F0E94F70F1C82DB
:101FC0001B821F5F143010F3198203C0002309F431
:101FD0000983F39454E05F1508F008CFDF91CF91A7
:101FE0001F910F91FF90EF90DF90CF900895DF92B7
:101FF000EF92FF920F931F93CF93DF93CDB7DEB78E
:1020000021970FB6F894DEBF0FBECDBF8983162F80
:10201000DD24833260F00D2D21E0AE014F5F5F4F74
:1020200067EC71E082E191E00E9469214EC09981E4
:1020300087E2989F700111248EE593E0E80EF91E67
:10204000F701868D9927807F9070803A910529F459
:102050000F2EF1E4DF2EF02D18C0F701868D9927A1
:10206000807F9070803B910529F40F2EF2E4DF2EE3
:10207000F02D0BC000E021E0AE014F5F5F4F63ED3C
:1020800071E082E191E00E946921112379F483E0FB
:10209000F701878380EF818387858F7B8787868D94
:1020A00042A16D2D8F700E94362D0FC0113069F442
:1020B000F70117828FE08183878586798787868DF0
:1020C00042A16D2D8F700E94812D21960FB6F8943C
:1020D000DEBF0FBECDBFDF91CF911F910F91FF905B
:1020E000EF90DF90089520E043EE58E067E270E063
:1020F0008170382F330FFA01E20FF11D8181823296
:1021000070F49927869FF001879FF00D969FF00D40
:102110001124EE59FC4F80818D7F832B80832F5FAC
:10212000203148F3089580915A0390915B030895FC
:102130008091590399270895EF92FF921F93CF93AF
:10214000DF937A018093D5086093D60810E0C12F01
:10215000DD27F701EC0FFD1F80810E94801C823279
:1021600020F4FE01EB52F74F82831F5F1C3078F39F
:10217000DF91CF911F91FF90EF9008959F92AF92C2
:10218000BF92CF92DF92EF92FF920F931F93CF9364
:10219000DF93CDB7DEB722970FB6F894DEBF0FBE40
:1021A000CDBF99240E94351E0E943E1F0E94691FC8
:1021B0008EEC98E00E94B61F1092C3081092C208DD
:1021C0009092C4089092C6089092C7089092C8084E
:1021D0009092C90882E1ECE8F8E011928A95E9F75B
:1021E0004EE958E028EB31E0892D9927880F991F97
:1021F000FC01E40FF51F31832083939461E169159D
:1022000098F799244CEF58E02DE030E0892D99277C
:10221000829FF001839FF00D929FF00D1124CF015A
:10222000E40FF51F11821482138216821582FC01BD
:10223000E450F74F8081846080839394F4E0F91533
:1022400028F70E94F627803221F487E68093110157
:1022500003C08EE6809311010F2EFEE5AF2EF3E052
:10226000BF2EF02D21E020935E0348EC50E0509308
:1022700071034093700332EA30937C0362EB609306
:102280007D03109280039FEF90937E0330937F0332
:1022900015E01093810383E0809382030F2EF7E211
:1022A000CF2EDD24F02DCA0CDB1C20938503F50115
:1022B00052AF41AFF601368F678F22A390A30F2E46
:1022C000F7EAFF2EF02DF1A213A38FE084A3F5010E
:1022D000E25BFF4F2093AC03538B428B0F2EF3EA4C
:1022E000EF2EF02DE68E83EB878F22A390A391A390
:1022F00093A389E084A3F501EB58FF4F2093D30308
:10230000538B428BF68E0F2EF7EBCF2EF02DC78E10
:1023100022A390A391A393A38BE084A3F501E45699
:10232000FF4F2093FA03538B428B0F2EF1EADF2EDF
:10233000F02DD68E81EB878F22A390A391A393A338
:102340008EE084A3F501ED53FF4F20932104538BBE
:10235000428B35EA368F05EB078F22A390A391A31A
:1023600093A38DE084A30F2EF6E09F2EF02DF501B0
:10237000E651FF4F20934804538B428B60EA668FEF
:1023800070EB778F12A290A331A313A394A2F5014F
:10239000EF5EFE4F20936F04538B428B368F078F77
:1023A00012A290A391A393A384E084A3F501E85C17
:1023B000FE4F20939604538B428B668F778F22A318
:1023C00090A361A313A38AE084A3F501E15AFE4F11
:1023D0002093BD04538B428B768F34EB378F12A33F
:1023E00090A391A393A382E184A3F501EA57FE4F42
:1023F0002093E404538B428B64EA668F378F22A3C9
:1024000090A3E1A213A388E084A3F501E355FE4F56
:1024100020930B05538B428B36EA368F86EB878FE2
:1024200012A290A361A313A324A30F2EFCE09F2E5E
:10243000F02DF501EC52FE4F20933205538B428B69
:10244000368F878F22A390A3D1A213A394A2F50164
:10245000E550FE4F20935905538B428BF68EC78E65
:1024600012A290A391A393A3CC246894C1F8C4A210
:102470009501F501EE5DFD4F71E070938005538B82
:10248000428BBD2CD68E0F2EF1EBEF2EF02DE78E6A
:1024900012A290A391A393A387E084A3F901E75B21
:1024A000FD4F7093A705538B428BE68EF02E078F5E
:1024B000612F12A390A391A393A381E184A3F901B7
:1024C000E059FD4F7093CE05538B428B14EA168F63
:1024D0000F2EF4EBDF2EF02DD78E12A290A386EAFA
:1024E00081A363A364A3F901E956FD4F7093F50539
:1024F000538B428B0F2EF3EAAF2EF02DA68E03EBFB
:10250000078F12A290A391A393A314A2F901E254FE
:10251000FD4F70E470931C064FEF5FEF538B428BBF
:10252000A7EAA68FD78E63E062A380A391A393A3AB
:1025300094A3F901EB51FD4F70934306538B428BEB
:10254000868FF78E62A380A391A393A394A3F9012E
:10255000E45FFC4F70936A06538B428B0F2EF5EAB3
:102560009F2EF02D968E86EB878F62A3A0A391A35A
:1025700093A394A3F901ED5CFC4F70939106538BE8
:10258000428B168F87EB878F62A3A0A391A393A39F
:1025900094A3F901E65AFC4F7093B806538B428B13
:1025A0000F2EF0EADF2EF02DD68E078F62A390A2B9
:1025B00091A393A394A3F901EF57FC4F7093DF0607
:1025C000538B428BB68EA2EBA78F62A390A291A3EE
:1025D00093A394A3F901E855FC4F70930607538B1E
:1025E000428B82EA868FE78E62A310A391A393A306
:1025F00094A3F901E153FC4F70932D07538B428B49
:10260000A68E80EB878F62A310A391A393A394A3BC
:10261000F901EA50FC4F70935407538B428BD68ECE
:10262000078FC2A2F0A291A393A394A3F901E35E42
:10263000FB4F70937B07538B428BB68EA78FC2A242
:10264000F0A291A393A3F901E35EFB4F94A3B90118
:10265000F901EC5BFB4FA0E4A093A207538B428BE4
:1026600082EA868FE78EC2A224EB20A391A393A3D4
:1026700094A3FB01E559FB4FA093C907538B428BF1
:10268000A68E80EB878FC2A220A391A393A394A3CD
:10269000FB01EE56FB4FA093F007538B428B87EA6A
:1026A000868F278FC2A226EB20A391A393A394A386
:1026B000FB01E754FB4FA0931708538B428B86EA2C
:1026C000868FF78EC2A220A391A393A394A3FB01AC
:1026D000E052FB4FA0933E08538B428B968E278F80
:1026E000C2A227EB20A391A393A394A3FB01E95FCC
:1026F000FA4FA0936508538B428B168F278FC2A287
:1027000020A391A393A394A3992447E250E02FE040
:10271000B92F06E11EE130E1892D9927849FF00150
:10272000859FF00D949FF00D1124CF017F01E60EDF
:10273000F71EF701158A148A168A8E599C4F9A83C0
:102740008983FC0180818C7F8083F7011786178A3B
:10275000218316A215A21686158614861386128664
:10276000B187E981FA8180818B7F8083F701108EA8
:1027700017820087168335832283128E118E148E62
:10278000138E158E9394F1E2F91530F622960FB65A
:10279000F894DEBF0FBECDBFDF91CF911F910F9197
:1027A000FF90EF90DF90CF90BF90AF909F900895F3
:1027B000ECE8F8E082E1DF011D928A95E9F7CF01AC
:1027C0000E94282720E06EE978E048EB51E0822F54
:1027D0009927880F991FFC01E60FF71F518340834B
:1027E0002F5F2231A0F38EE998E00E9448270895D8
:1027F000AF92BF92CF92DF92EF92FF920F931F930F
:10280000CF93DF93CDB7DEB7C656D0400FB6F8945E
:10281000DEBF0FBECDBFDD240F2EF5E1EF2EFF246E
:10282000F02DEC0EFD1E2D2D332787E290E0289F22
:10283000A001299F500D389F500D1124FA01E25A32
:10284000FC4F82899389892F99278D8B82898E8B62
:1028500086818F8B1A8E198E1B8E8581888F80853D
:102860008C8F8FE0D89EC001112487539C4FBC01F0
:10287000CE014D960E94C0511CA68FEF8DA71D2D35
:102880001F5F612FC7010E944626A895D12E51E2F5
:10289000511748F684E688AB88E789AB4CE050E0F6
:1028A0006FEF70E0CE01C2960E94D451CE01C09667
:1028B0000E94862481EC8EAF40E150E06FEF70E023
:1028C000CE01CF960E94D451CE01CE960E94B42460
:1028D000A895DD240F2EF4E1CF2EF02D7E01089473
:1028E000E11CF11C0FE0D701EC2D1D92EA95E9F7F0
:1028F000D09EC00111248C5D9C4FBC01C7010E9479
:10290000C051188A1D2D1F5FB701812F0E94DD263F
:10291000D12EFAE0F11738F7A895DD240F2EF8E54F
:10292000AF2EBB24F02DAC0EBD1E0F2EFFE0EF2E00
:10293000F02D8E01015B1F4FFF24FA94D501EE2D7F
:102940001D92EA95E9F7DE9CC001112487529D4F44
:10295000BC01C80109960E94C051D8011C92F8011F
:102960001182128281E083838AE084838081F8016E
:10297000E80FF11DF5828F5F8430C8F3BE01615B03
:102980007F4F8D2D0E94F424D394F4E0FD15B0F612
:10299000E4EFF8E088E0DF011D928A95E9F7CF01C6
:1029A0000E94D4240E94311FCA59DF4F0FB6F894F9
:1029B000DEBF0FBECDBFDF91CF911F910F91FF9072
:1029C000EF90DF90CF90BF90AF9008950F931F933B
:1029D000CF93DF93CDB7DEB7E3970FB6F894DEBFA2
:1029E0000FBECDBF00E0102F1F5F612FCE010196FB
:1029F0000E948B26202F332787E290E0289FA0019A
:102A0000299F500D389F500D1124FA01E25AFC4FB6
:102A100089819927982F88272A81820F911D938B6E
:102A2000828B8B818683888580878C818583888D46
:102A30008487898D81878D819E81928F818F8F81FF
:102A4000858F012F123278F285ED98E00E94A42440
:102A500083EE98E00E94C4248CE898E00E94382716
:102A60008EE998E00E94582784EF98E00E94E424C1
:102A70000E94311F00E0BE01645E7F4F802F0E94E4
:102A80002D25202F33278DE090E0289FA001299F3E
:102A9000500D389F500D11249A01FA01E450F74F60
:102AA0008C8D582F51708081482F4C7F8D8D817077
:102AB000982F990F842F852B892B8083F901E4505F
:102AC000F74F8E8D82838F8D878388A18087F90150
:102AD000EB5FF64F89A19AA1ABA1BCA18083918342
:102AE000A283B3830F5F053030F2E3960FB6F894FC
:102AF000DEBF0FBECDBFDF91CF911F910F91089523
:102B0000CF93DF93EC01862F0E94801C8332D8F490
:102B1000282F332787E290E0289FA001299F500D9E
:102B2000389F500D1124FA01E25AFC4F8F89848797
:102B300088819927982F88272981820F911D938B4F
:102B4000828B8A818683DF91CF9108959091E308EB
:102B5000892F8150853168F4892F0E94470A882384
:102B600021F081E00E947310089580E00E947310AC
:102B700008959091E308892F86518F3068F4892F4A
:102B80000E942C45882321F081E00E947310089553
:102B900080E00E94731008958091E3080E94B03491
:102BA0008E3F41F0813019F40E947310089580E047
:102BB0000E9473100895FC0184818860848380EFF3
:102BC0008283878586798787178A168A848525E098
:102BD000829FC001112496878587892B41F48185C6
:102BE0008F3F29F0829FC00111249387828783E061
:102BF000878308951F93CF93C0E017E2C19FC00160
:102C00001124FC01E25AFC4F8785992783FD02C0FD
:102C100080FF03C0CF010E94DB15CF5FC23270F38B
:102C2000CF911F910895FF920F931F93CF93DF933E
:102C300010E00F2EFFE0FF2EF02D82E00E943035D5
:102C400087E2189FC0011124EC01C25ADC4F88852D
:102C5000882361F48981803F09F0CCC08C81886031
:102C60008C838F85867B8F87FA82C4C02885822FCC
:102C700081508531D0F58F85992783FD24C080FD53
:102C800022C0822F0E94470A882341F089818F3019
:102C900009F0B0C0CE010E94DB15ACC08981803F35
:102CA00009F0A8C089858F3F09F4A4C08A859B8557
:102CB000892B09F09FC08C8188608C838F85867BEF
:102CC0008F87FA8297C088850E94470A882309F077
:102CD00091C08981803F09F08DC08C8188608C8390
:102CE0008F85867B8F87FA8285C02885822F8651C3
:102CF0008A30D0F58F85992783FD24C080FD22C0BE
:102D0000822F0E942C45882341F089818F3009F061
:102D100071C0CE010E94DB156DC08981803F09F032
:102D200069C089858F3F09F465C08A859B85892B99
:102D300009F060C08C8188608C838F85867B8F874B
:102D4000FA8258C088850E942C45882309F052C019
:102D50008981803F09F04EC08C8188608C838F858B
:102D6000867B8F87FA8246C000E088850E94B03457
:102D7000982F8E3FA9F08885803C21F49130A1F4F2
:102D8000092F12C08D81813021F4913011F4092F67
:102D90000BC08D81803141F4992331F401E004C0EE
:102DA00088858F3F09F401E0002369F089818F3025
:102DB00009F58F85992783FD1DC080FD1BC0CE01BD
:102DC0000E94DB1517C08981803F31F08F859927DC
:102DD00083FD02C080FF0EC089858F3F59F08A8530
:102DE0009B85892B39F48C8188608C838F85867BC9
:102DF0008F87FA821F5F123208F41FCFDF91CF91C5
:102E00001F910F91FF900895609358030895CF93F9
:102E1000DF93EC0188818150823218F080E090E0ED
:102E200036C088810E94801C282F898199278F3085
:102E3000910521F0803F9105A1F027C0332787E25B
:102E400090E0289FA001299F500D389F500D11241C
:102E5000FA01E25AFC4F8FE081838785867F87875E
:102E600014C0332787E290E0289FA001299F500DCE
:102E7000389F500D1124FA01E25AFC4F80EF8183F4
:102E80008785867F8787178A168A81E090E0DF91A1
:102E9000CF9108958F929F92AF92BF92CF92DF927F
:102EA000EF92FF920F931F93CF93DF93CDB7DEB7CF
:102EB00021970FB6F894DEBF0FBECDBFBB24B982F9
:102EC0008B2CAB2C9B2C1092C3081092C208B09292
:102ED000C608B092C808B092C7080E94A4048093A4
:102EE000C50880915803882309F085C2B9828B2DCB
:102EF000823208F0D0C482E00E9430358824998163
:102F000087E2989FC00111240F2EFEE5CF2EF3E03B
:102F1000DF2EF02DC80ED91EF601868D9927807FF1
:102F20009070803A910529F40F2EF1E4AF2EF02D28
:102F300018C0F601868D9927807F9070803B91059F
:102F400029F40F2EF2E4AF2EF02D0BC000E021E0AB
:102F5000AE014F5F5F4F66E276E082E191E00E9452
:102F60006921F601118A108A248122FDCEC0808158
:102F700099278130910509F466C08034910509F0E4
:102F8000D1C0818199278F309105B1F1803F9105A2
:102F900009F0C8C0822F837019F4878585FF09C0A6
:102FA000F601868D42A16A2D8F700E94812D8824A2
:102FB00010C0F60185859685892B59F4878580FD9B
:102FC00008C0868D42A16A2D8F700E94362D8824FC
:102FD0008394F601848183FFA5C0877F84838281E7
:102FE0008F3009F09FC08183868D42A16A2D8F703A
:102FF0000E94812D882496C0F601248123FF1AC0E7
:10300000822F877F84838281803F09F08BC08183F8
:1030100085859685892B09F085C0822F837009F0FC
:1030200081C0868D42A16A2D8F700E94362D882422
:10303000839478C0F601868D42A16A2D8F700E941C
:10304000812D88246FC0F601818199278F309105E9
:10305000C1F1803F910509F065C08481837019F446
:10306000878585FF09C0F601868D42A16A2D8F7084
:103070000E94812D882413C0F60185859685892BB1
:1030800071F48785992780FD0AC083FD08C0868D6D
:1030900042A16A2D8F700E94362D88248394F601F8
:1030A000848183FF3FC0877F848382818F30D1F505
:1030B0008183868D42A16A2D8F700E94812D882484
:1030C00031C0F601248123FF17C0822F877F8483BC
:1030D0008281803F39F5818385859685892B11F51D
:1030E000822F8370F9F4868D42A16A2D8F700E9421
:1030F000362D8824839416C0F601868D42A16A2D50
:103100008F700E94812D88240DC0F601818199273E
:103110008F30910531F0803F910521F4882483940C
:1031200001C08824F6018181803F09F058C084A144
:103130008F3F09F454C00E9473037C0100271127BC
:10314000F601F6A2E5A289819927FC01E457F74F21
:1031500080819927AA27BB278E159F05A007B10755
:1031600024F0EE24FF2487010AC089819927FC01FD
:10317000E457F74F8081E81AF10801091109F3E0DB
:10318000EF16F10401051105CCF089819927880F0C
:10319000991FFC01E256F74F808191819C014427E1
:1031A0005527C801B7010E94E55120EE31E040E00B
:1031B00050E00E94595279018A0103C0EE24FF2495
:1031C0008701F601F18AE08A8091C2089091C308D4
:1031D0008E0D9F1D9093C3088093C20803C0F60113
:1031E000118A108A882039F4F601838D948D892BF9
:1031F00011F0148E138EF60187859927AC01487063
:10320000507083FD66C02089318982899389821735
:103210009307A0F5838D948D892B11F0548F438FE4
:10322000F60186898130F9F484899589892B09F022
:1032300050C08785886087878091C6088F5F80939C
:10324000C6088081813039F4868D42A16A2D8F7045
:103250000E94812D88248981F601608971898F5FA0
:103260000E94DC2336C081E0F601868B968185E0E2
:10327000989FC0011124958B848B2BC0F601168A70
:10328000218D328D2115310521F18820A1F0808911
:1032900091898217930778F4838D948D892BC9F4D3
:1032A000878586FD16C0958D85E0989FC001112405
:1032B000948F838F0EC0F601838D948D892B49F0F6
:1032C00020893189818D928D8217930710F4148E95
:1032D000138EF601878D9927807F9070803A910533
:1032E00029F40F2EF1E49F2EF02D18C0F601878DE2
:1032F0009927807F9070803B910529F40F2EF2E48E
:103300009F2EF02D0BC000E021E0AE014F5F5F4F1C
:1033100066E477E082E191E00E946921F601878D01
:1033200042A1692D8F700E94042E282FF601818101
:10333000803F09F043C08785992783FD3FC080FD0A
:103340003DC09091C508809111018917B8F5F1E051
:103350008F1691F5222381F5F6018781882371F577
:103360008485882359F5808D8F3F11F08F5F808F82
:10337000F601808D863010F187898F5F878B8431CD
:1033800058F4868D42A16A2D8F700E94812DF6011E
:10339000108E83E0878312C0F601868D42A16A2DCC
:1033A0008F700E94812DF6018785816087878981D2
:1033B0008F5F0E94142402C0F601108EF6018785EB
:1033C00080FF05C08091C8088F5F8093C808F60110
:1033D000878583FF05C08091C6088F5F8093C608EC
:1033E000F60187858111B39489818F5F8983823249
:1033F00008F481CD50C280915803813009F09CC1FE
:1034000019828981982F823208F045C287E2989FFD
:10341000C00111240F2EFEE5CF2EF3E0DF2EF02D9C
:10342000C80ED91EF601868D9927807F9070803A4C
:10343000910529F40F2EF1E4AF2EF02D0CC0F6010A
:10344000868D9927807F9070803B910521F40F2E07
:10345000F2E4AF2EF02DF601848182FD4FC0808111
:1034600099278130910569F18034910509F046C0B2
:10347000818199278F30910561F0803F9105F1F5A9
:10348000868D42A16A2D8F700E94362D88248394E8
:1034900035C08981282F332787E290E0289FA0013B
:1034A000299F500D389F500D1124FA01E25AFC4F0C
:1034B000868DF60142A16A2D8F700E94812D88248D
:1034C0001DC0F601818199278F30910561F0803F01
:1034D0009105A1F4868D42A16A2D8F700E94362D30
:1034E000882483940BC0F601868D42A16A2D8F70CB
:1034F0000E94812D8FE0F60181838824F60181816D
:10350000803F09F057C084A18F3F09F453C00E9447
:1035100073037C0100271127F601F6A2E5A2898139
:103520009927FC01E457F74F80819927AA27BB27E9
:103530008E159F05A007B10724F0EE24FF24870114
:103540000AC089819927FC01E457F74F8081E81A66
:10355000F10801091109F3E0EF16F1040105110565
:10356000CCF089819927880F991FFC01E256F74F0B
:10357000808191819C0144275527C801B7010E9491
:10358000E55120EE31E040E050E00E9459527901CF
:103590008A0103C0EE24FF248701F601F18AE08A44
:1035A0008091C2089091C3088E0D9F1D9093C3080F
:1035B0008093C208F6012089318982899389821714
:1035C000930780F58689813011F584899589892B47
:1035D00069F58785886087878091C6088F5F8093AB
:1035E000C6088081813059F4868D42A16A2D8F7082
:1035F0000E94812D88248FE0F60181838283898156
:10360000F601608971898F5F0E94DC230FC081E021
:10361000F601868B968185E0989FC0011124958BD9
:10362000848B04C0F601168A158A148AF601878DE8
:103630009927807F9070803A910529F40F2EF1E44C
:103640009F2EF02D0CC0F601878D9927807F9070FA
:10365000803B910521F40F2EF2E49F2EF02DF60110
:10366000878D42A1692D8F700E94042E282FF601AC
:103670008785992783FD42C080FD40C09091C50891
:10368000809111018917D0F5F1E08F16A9F5222359
:1036900099F5F6018781882389F58485882371F55A
:1036A0008181803F59F5808D8F3F11F08F5F808F32
:1036B000F601808D863010F187898F5F878B84318A
:1036C00058F4868D42A16A2D8F700E94812DF601DB
:1036D000108E83E0878312C0F601868D42A16A2D89
:1036E0008F700E94812DF60187858160878789818F
:1036F0008F5F0E94142402C0F601108EF6018785A8
:1037000080FF05C08091C8088F5F8093C808F601CC
:10371000878583FF05C08091C6088F5F8093C608A8
:10372000F60187858111B39489818F5F8983982FF2
:10373000823208F46BCEAFC080915803823009F01A
:10374000AAC019828981982F823208F0A4C087E22A
:10375000989FC00111240F2EFEE5CF2EF3E0DF2E3F
:10376000F02DC80ED91EF601868D9927807F9070A6
:10377000803A910529F40F2EF1E4AF2EF02D0CC004
:10378000F601868D9927807F9070803B910521F40A
:103790000F2EF2E4AF2EF02DF601868D42A16A2D98
:1037A0008F700E94362DF60184A18F3F09F46CC002
:1037B0000E9473037C0100271127F601F6A2E5A2FF
:1037C0008091570380FF1CC089819927FC01E45731
:1037D000F74F80819927AA27BB278E159F05A00741
:1037E000B10724F0EE24FF2487010AC089819927BC
:1037F000FC01E457F74F8081E81AF108010911092B
:10380000F3E0EF16F1040105110574F180915703FF
:1038100081FF19C089819927880F991FFC01E25601
:10382000F74F808191819C0144275527C801B7013A
:103830000E94E55120EE31E040E050E00E945952F4
:1038400079018A0114C0C801B70128EB31E040E0DA
:1038500050E00E94E55120EE31E040E050E00E944F
:10386000595279018A0103C0EE24FF248701F60131
:10387000F18AE08A8091C2089091C3088E0D9F1D45
:103880009093C3088093C20889818F5F8983982FA2
:10389000823208F45CCFBB2031F4B092C708B092FA
:1038A000C808B092C9080E949804982F8093C40851
:1038B00080915903891710F4909359032091C208FD
:1038C0003091C30880915A0390915B03821793074C
:1038D00020F430935B0320935A0321960FB6F8949B
:1038E000DEBF0FBECDBFDF91CF911F910F91FF9033
:1038F000EF90DF90CF90BF90AF909F908F90089502
:10390000815099270895CF93DF93EC01862F0E9471
:10391000801C833278F4282F332787E290E0289F99
:10392000A001299F500D389F500D1124FA01E25A31
:10393000FC4FC683DF91CF910895EF92FF921F93C2
:10394000CF937C01C0E080EC0E94B0348111C1E0D3
:1039500081EC0E94B0348111C26082EC0E94B034CC
:103960008111C46081ED0E94B0348111C86084EC83
:103970000E94B0348111C06185EC0E94B034811185
:10398000C06286EC0E94B0348111C06487EC0E9452
:10399000B0348111C06810E083EC0E94B034811112
:1039A00011E082ED0E94B0348111126083ED0E941B
:1039B000B03481111460F701C0831183C0E081E04D
:1039C0000E94470A8111C1E082E00E94470A8111EA
:1039D000C26083E00E94470A8111C46084E00E94B3
:1039E000470A8111C86085E00E94470A8111C061C1
:1039F00086E00E94470A8111C06287E00E94470A60
:103A00008111C06488E00E94470A8111C068F701F3
:103A1000C283C0E089E00E94470A8111C1E08AE0C8
:103A20000E94470A8111C2608BE00E94470A8111FF
:103A3000C4608CE00E94470A8111C8608DE00E943A
:103A4000470A8111C0618EE00E94470A8111C0625D
:103A50008FE00E94470A8111C06480E10E94470AFA
:103A60008111C068F701C383C0E081E10E94470A69
:103A70008111C1E082E10E94470A8111C26083E1A5
:103A80000E94470A8111C46084E10E94470A8111A3
:103A9000C86085E10E94470A8111C061F701C483B3
:103AA000CF911F91FF90EF9008951F93CF93DF93D5
:103AB000182FEB010E94801C482F833218F080E001
:103AC00090E06FC0992727E230E0829FB001839F8A
:103AD000700D929F700D1124FB01EE59FC4F208157
:103AE00022FD20C0FB01E25AFC4F8181803F51F44E
:103AF00021FD05C020FD03C0878585FF03C08FE041
:103B0000888335C0242F332787E290E0289FF00177
:103B1000299FF00D389FF00D1124E25AFC4F81814E
:103B2000888325C030E0232F5DE0259FC00111244C
:103B3000DC01A450B74FFD018181813099F490E000
:103B40007FE060EFFD01E90FF11D8185841739F4F5
:103B500031E08C9182FF02C0788301C068839F5F4F
:103B6000943080F32F5F253010F43323F1F2242FAB
:103B7000332787E290E0289FA001299F500D389FAE
:103B8000500D1124FA01E25AFC4F87858983808900
:103B900091899C838B83812F0E945F248A8381E09B
:103BA00090E0DF91CF911F9108950E94801C833295
:103BB00018F080E090E00895282F332787E290E006
:103BC000289FA001299F500D389F500D1124FA0104
:103BD000E25AFC4F8181803F59F4FA01EE59FC4FC3
:103BE000208121FD05C020FD03C081E090E0089503
:103BF00080E090E008950E94801C833218F080E0FD
:103C000090E00895282F332787E290E0289FA001B5
:103C1000299F500D389F500D1124FA01E25AFC4F94
:103C20002785283011F0213019F481E090E00895C3
:103C300080E090E00895FC018091C2089091C30853
:103C4000918380838091C40882838091C508838397
:103C50008091C60884838091C70885838091C808B5
:103C600086838091C908878308959EEF81B1892357
:103C700081B982B1892382B917B818B891EF8AB196
:103C800089238AB98BB189238BB908950F930E9438
:103C9000801C282F833168F000E0202F40E050E0A6
:103CA0006DEB79E082E191E00E94692180E090E093
:103CB00007C08CE898E0FC01E20FF11D8081992794
:103CC0000F9108950F930E94801C833168F000E0EB
:103CD000202F40E050E06BEC79E082E191E00E941F
:103CE000692180E692E212C09927880F991FFC0192
:103CF000E256F74F2081318184E190E0289FA001B6
:103D0000299F500D389F500D1124CA010F9108951D
:103D10000F93CF93DF93EB010E94801C833158F007
:103D200000E0202F40E050E06AED79E082E191E090
:103D30000E94692112C099272EE938E0880F991F47
:103D4000FC01E20FF31FCE0164E170E00E9410520B
:103D500071836083C9010E944827DF91CF910F9141
:103D600008950E94801C833118F080E090E008954F
:103D7000282F332787E290E0289FA001299F500D2C
:103D8000389F500D1124FA01E25AFC4F8089918925
:103D900008950E94801C833118F080E090E008951F
:103DA000282F332787E290E0289FA001299F500DFC
:103DB000389F500D1124FA01E25AFC4F85A196A1BB
:103DC00008958093570308950F931F93CF93DF9324
:103DD00010E0012F87E2189FC0011124EC01C25AA4
:103DE000DC4F8E8D9927807F9070803A910511F479
:103DF00001E408C08E8D9927807F9070803B9105EB
:103E000009F402E48E8D4AA1602F8F700E94362D36
:103E10008CA18F3F41F00E947303212F3327F901BA
:103E2000E457F74F80831F5F1231A0F28CE898E0CF
:103E30000E942827DF91CF911F910F910895CF9372
:103E400080915803833059F083E080935803C0E099
:103E500061E08C2F0E94F70FCF5FC232C8F3CF9181
:103E600008958091F508882341F00E943E1F0E942A
:103E7000691F8EEC98E00E94B61F0895259A2D9830
:103E8000269A2E988AEA8093800089E180938100A7
:103E9000109285001092840080E395E09093870053
:103EA00080938600109289001092880010928B00F7
:103EB00010928A0010928D0010928C0060E070E0E9
:103EC00081E00E94941F60E070E082E00E94941FF5
:103ED00008951092900084E08093910010929500D4
:103EE00010929400109297001092960010929900F0
:103EF0001092980010929B0010929A0010929D00D0
:103F000010929C001092CB081092CA081092CD0813
:103F10001092CC08809169008860809369001092AB
:103F20006A00E99AE19A089599278230910581F013
:103F3000833091051CF4019721F00895039779F0DF
:103F40000895872F992780938900609388000895AA
:103F5000872F992780938B0060938A000895872F7D
:103F6000992780938D0060938C000895FC01118245
:103F700010821382128285E090E0958384831682FA
:103F80000895EF92FF920F931F93CF93DF93EC016D
:103F90008E81982F8F5F8E83963068F060E375E096
:103FA00081E00E94941F60E375E082E00E94941F0C
:103FB00086E08E8355C08A819B819C0144275527CA
:103FC000888199817C0100271127DA01C901689451
:103FD00012F8880F991FAA1FBB1F1694D1F7820FE2
:103FE000931FA41FB51F280F391F4A1F5B1FCA014B
:103FF000B90125E830E040E050E00E94E551A80119
:1040000097010E943752E901C901845490408652B9
:10401000944010F0C0E3D5E08091F508882349F082
:1040200080912204803F29F4BE0181E00E94941F08
:1040300005C060E375E081E00E94941F8091F6085E
:10404000882349F080915A05803F29F4BE0182E01F
:104050000E94941F05C060E375E082E00E94941FF7
:10406000DF91CF911F910F91FF90EF9008951F92D4
:104070000F920FB60F9211242F933F938F939F931C
:1040800080919400282F3327322F2227809195008A
:104090009927282B392B8091690099278C70907073
:1040A0000C97E1F43093CF082093CE08109294003F
:1040B0001092950080915C0390915D039093D108DC
:1040C0008093D00810925D0310925C031092D40884
:1040D000809169008B7F8093690010C08091690096
:1040E00099278C709070089749F430935D03209362
:1040F0005C03809169008460809369009F918F9137
:104100003F912F910F900FBE0F901F901895CF9356
:10411000DF93CDB7DEB723970FB6F894DEBF0FBE9F
:10412000CDBFFE013196A0E8B1E083E090E021E050
:104130008030920719F40E94B35203C0182E0E94D7
:10414000B35243E050E060E271E0CE0101960E947C
:104150002D42882391F00E94C720E0E2F1E0A0E820
:10416000B1E083E090E021E08030920719F40E94F2
:10417000C45203C0182E0E94C452279823960FB62B
:10418000F894DEBF0FBECDBFDF91CF910895CF93DE
:10419000DF93CDB7DEB76E970FB6F894DEBF0FBED4
:1041A000CDBF84E1FE013B9611928A95E9F720E0AC
:1041B00064E144E150E0342FFE013B96269FC001AC
:1041C0001124DC01AC57BE4F4115510551F081E07F
:1041D0004030580719F40E94C45203C0132E0E94A5
:1041E000C452A8952F5F2C3038F31982FE01319606
:1041F000A3E8B1E081E090E021E08030920719F47B
:104200000E94C45203C0182E0E94C4526E960FB66C
:10421000F894DEBF0FBECDBFDF91CF910895CF934D
:10422000DF93CDB7DEB721970FB6F894DEBF0FBE90
:10423000CDBFFE013196A3E8B1E081E090E021E03E
:104240008030920719F40E94B35203C0182E0E94C6
:10425000B35289818D3010F08CE089838981992750
:1042600021960FB6F894DEBF0FBECDBFDF91CF9180
:104270000895CF93DF93CDB7DEB764970FB6F89468
:10428000DEBF0FBECDBF9B01FE01319694E1899F39
:10429000D0011124A059BE4F84E190E041E080306C
:1042A000940719F40E94B35203C0182E0E94B3520F
:1042B00084E1FE013196D90101900D928A95E1F7D2
:1042C00064960FB6F894DEBF0FBECDBFDF91CF91DD
:1042D00008956F927F928F929F92AF92BF92CF92EA
:1042E000DF92EF92FF920F931F93CF93DF93CDB79F
:1042F000DEB7A9970FB6F894DEBF0FBECDBF6C0135
:104300005B013A01022FFE01B996A3E8B1E081E01A
:1043100090E021E08030920719F40E94B35203C06C
:10432000182E0E94B35289A58C3008F0D4C099246D
:10433000FE01759684E1DF011D928A95E9F7B601C9
:10434000CF010E94DE51192D89A5981608F05EC094
:104350000F2EF4E18F2EF02D0F2EF4E1EF2EFF241F
:10436000F02DFE013196189DC0011124DC01AC57DF
:10437000BE4FE114F10459F020E0E21621E0F2060C
:1043800019F40E94B35203C01E2C0E94B3528D85B3
:104390009E858A159B0599F546E050E0B601CE0151
:1043A00001960E942D42882351F5992493948F857C
:1043B0008A3008F090C0890D8F87053008F004E03E
:1043C000198A1A8A1B8A1C8A802F9927AC01B3018B
:1043D000CE0141960E94C751FE013196189DD00131
:1043E0001124AC57BE4F84E190E021E08030920769
:1043F00019F40E94C45203C0182E0E94C4521F5FB9
:1044000089A5181718F4992009F4ABCF992009F061
:1044100052C089A58C3008F04EC08F5F89A78CE010
:10442000FE01319611928A95E9F7F601019000207C
:10443000E9F731972E2F2C192C3008F02BE010E0E3
:10444000121780F4AE014F5F5F4F812F9927DC0177
:10445000A40FB51FF601E80FF91F80818C931F5F31
:10446000121798F3BE86AD8681E08F87053008F07D
:1044700004E0088B198A1A8A1B8A1C8A802F9927C4
:10448000AC01B301CE0141960E94C751FE013196A5
:1044900099A584E1989FD0011124A059BE4F84E1D1
:1044A00090E021E08030920719F40E94C45203C0CA
:1044B000182E0E94C452FE01B996A3E8B1E081E033
:1044C00090E021E08030920719F40E94C45203C0AA
:1044D000182E0E94C452A9960FB6F894DEBF0FBEE4
:1044E000CDBFDF91CF911F910F91FF90EF90DF90A3
:1044F000CF90BF90AF909F908F907F906F900895D6
:10450000089582E1E5EBFDE011928A95E9F780E1FB
:10451000E7ECFDE011928A95E9F7E9EEFDE0A8E805
:10452000B0E082E190E021E08030920719F40E942F
:10453000B35203C0182E0E94B352EBEFFDE0AAE97C
:10454000B0E082E190E021E08030920719F40E940F
:10455000B35203C0182E0E94B352EDE0FEE0ACEA65
:10456000B0E080E190E021E08030920719F40E94F1
:10457000B35203C0182E0E94B352E7EDFDE0ADEB3D
:10458000B0E082E190E021E08030920719F40E94CF
:10459000B35203C0182E0E94B352EDE3F9E0A5E830
:1045A000B0E081E090E021E08030920719F40E94B1
:1045B000B35203C0182E0E94B352EEE3F9E0A6E80E
:1045C000B0E082E090E021E08030920719F40E9490
:1045D000B3520895182E0E94B3520895CF93DF93DB
:1045E000CDB7DEB762970FB6F894DEBF0FBECDBF72
:1045F000FE01319682E1DF011D928A95E9F7A8E874
:10460000B0E082E190E021E08030920719F40E944E
:10461000C45203C0182E0E94C452FE013196AAE96A
:10462000B0E082E190E021E08030920719F40E942E
:10463000C45203C0182E0E94C452FE013196ACEA47
:10464000B0E080E190E021E08030920719F40E9410
:10465000C45203C0182E0E94C452FE013196ADEB25
:10466000B0E082E190E021E08030920719F40E94EE
:10467000C45203C0182E0E94C4520E948122629626
:104680000FB6F894DEBF0FBECDBFDF91CF91089576
:104690000E949810982F80913D09891790F490936B
:1046A0003D09EDE3F9E0A5E8B0E081E090E021E02C
:1046B0008030920719F40E94C45203C0182E0E9441
:1046C000C4520E9493109C0180913E0990913F0931
:1046D00082179307A0F430933F0920933E09EEE33D
:1046E000F9E0A6E8B0E082E090E021E080309207B7
:1046F00019F40E94C4520895182E0E94C4520895BD
:1047000080913D099927089580913E0990913F0934
:10471000089590E045EB5DE0292F3327F901E40F80
:10472000F51F808180FF17C08E7F8083D901A85735
:10473000BF4FF901E751F24F8081082E0E94B85215
:10474000D901A656BF4FF901E550F24F8081082EDE
:104750000E94B8520895E92FFF27DF01A40FB51F6B
:104760008C9181FF0CC08D7F8C93DF01A354BF4FD0
:10477000E952F24F8081082E0E94B85208959F5F3F
:10478000923150F290E027EC3DE0E92FFF27DF0166
:10479000A20FB31F8C91813059F41C92DF01A455F4
:1047A000BF4FE35FF14F8081082E0E94B8520895F9
:1047B0009F5F903150F30895282F2150223198F5B2
:1047C00089EE9DE0FC01E20FF11D3081832F9927D6
:1047D000929582958F7089279F7089278F309105D8
:1047E00014F5482F4F5F942F9295907F832F8F70F1
:1047F000890F8083CB0183709070892B11F041E089
:1048000001C040E03327F901E550F24FCB01969506
:10481000879596958795840F8083F901EB54F24F25
:104820008081816080830895E82FE150E231C0F4F7
:10483000FF27DF01A751B24F2C91822F99278F704C
:1048400090700F971CF5822F8F708F5F922F907F43
:10485000890F8C93EB54F24F80818160808308959F
:104860008351803198F4E82FFF27DF01A35FB14F18
:104870002C91822F99278F7090700F973CF4822F84
:104880008F5F8C93E953F24F81E0808308958150CC
:104890008231A0F4E82FFF27DF01A952B24F2C91FB
:1048A000822F99278F7090700F9744F4822F8F5F1B
:1048B0008C93EB54F24F8081826080830895E82FBF
:1048C000E150E23188F42E2F3327F901E751F24FFE
:1048D0008081882331F4F901E952F24F80818823E5
:1048E00091F081E090E00895282F2351203158F471
:1048F0008DE09EE0FC01E20FF11D8081882319F01C
:1049000081E090E0089580E090E00895CF93DF93F8
:10491000EC01FC0120EA32E08EE090E041E08030E2
:10492000940721F4D9010E94C45204C0D901182E61
:104930000E94C452CE010296AC01698188810E9416
:104940009C10DF91CF910895FC01A0EAB2E08EE0C7
:1049500090E021E08030920719F40E94B35208954C
:10496000182E0E94B3520895FC01A0EBB2E081E141
:1049700090E021E08030920719F40E94C45208951B
:10498000182E0E94C4520895FC01A0EBB2E081E110
:1049900090E021E08030920719F40E94B35208950C
:1049A000182E0E94B3520895FC01A0EFB9E088E0F0
:1049B00090E021E08030920719F40E94C4520895DB
:1049C000182E0E94C4520895FC01A0EFB9E088E0BF
:1049D00090E021E08030920719F40E94B3520895CC
:1049E000182E0E94B35208950F93CF93DF93CDB743
:1049F000DEB721970FB6F894DEBF0FBECDBF898317
:104A0000853060F000E021E0AE014F5F5F4F67E46A
:104A100070E084E291E00E94692115C0898198E1EB
:104A2000899FC0011124FB01DC01A053B24F88E132
:104A300090E021E08030920719F40E94C45203C034
:104A4000182E0E94C45221960FB6F894DEBF0FBEF6
:104A5000CDBFDF91CF910F9108950F93CF93DF9347
:104A6000CDB7DEB721970FB6F894DEBF0FBECDBF2E
:104A70008983853060F000E021E0AE014F5F5F4F39
:104A800064E570E084E291E00E94692115C08981AB
:104A900098E1899FC0011124FB01DC01A053B24FB2
:104AA00088E190E021E08030920719F40E94B3522F
:104AB00003C0182E0E94B35221960FB6F894DEBFA1
:104AC0000FBECDBFDF91CF910F9108950F93CF937C
:104AD000DF93CDB7DEB721970FB6F894DEBF0FBED8
:104AE000CDBF8983853160F000E021E0AE014F5FEA
:104AF0005F4F60E670E084E291E00E94692114C09B
:104B0000FB0199818CE2989FD0011124A053BC4FE6
:104B10008CE290E021E08030920719F40E94C452A8
:104B200003C0182E0E94C45221960FB6F894DEBF1F
:104B30000FBECDBFDF91CF910F9108950F93CF930B
:104B4000DF93CDB7DEB721970FB6F894DEBF0FBE67
:104B5000CDBF8983853160F000E021E0AE014F5F79
:104B60005F4F6AE670E084E291E00E94692114C020
:104B7000FB0199818CE2989FD0011124A053BC4F76
:104B80008CE290E021E08030920719F40E94B35249
:104B900003C0182E0E94B35221960FB6F894DEBFC0
:104BA0000FBECDBFDF91CF910F9108950F93CF939B
:104BB000DF93CDB7DEB721970FB6F894DEBF0FBEF7
:104BC000CDBF89838F3060F000E021E0AE014F5F00
:104BD0005F4F64E770E084E291E00E94692114C0B5
:104BE000FB01998189E1989FD0011124A056B84F0B
:104BF00089E190E021E08030920719F40E94C452CC
:104C000003C0182E0E94C45221960FB6F894DEBF3E
:104C10000FBECDBFDF91CF910F9108950F93CF932A
:104C2000DF93CDB7DEB721970FB6F894DEBF0FBE86
:104C3000CDBF89838F3060F000E021E0AE014F5F8F
:104C40005F4F6EE770E084E291E00E94692114C03A
:104C5000FB01998189E1989FD0011124A056B84F9A
:104C600089E190E021E08030920719F40E94B3526C
:104C700003C0182E0E94B35221960FB6F894DEBFDF
:104C80000FBECDBFDF91CF910F910895CF93DF93EA
:104C9000CDB7DEB76B970FB6F894DEBF0FBECDBFB2
:104CA000FC01862F8150823218F080E090E02AC00B
:104CB00061508081898381818A8382818B83838112
:104CC0008C83878188878789888F808D898F84816D
:104CD00095819E838D8386818F83DF0118968FE077
:104CE000FE0139960D9001928A95E1F78BE1689F5C
:104CF000C00111248050964FBC01CE0101960E9444
:104D0000172799276B960FB6F894DEBF0FBECDBF5D
:104D1000DF91CF9108950F931F93CF93DF93CDB77A
:104D2000DEB76B970FB6F894DEBF0FBECDBF8C0118
:104D3000962F91509232B0F58BE1989FC0011124CB
:104D40009E012F5F3F4FDC01A050B64F8BE190E0FA
:104D500041E08030940721F4F9010E94B35204C06D
:104D6000F901182E0E94B3528981F80180838A814B
:104D700081838B8182838C81838388858783888DDF
:104D8000878B898D808F8D819E81958384838F8190
:104D90008683D80118968FE0FE01399601900D9216
:104DA0008A95E1F76B960FB6F894DEBF0FBECDBFC4
:104DB000DF91CF911F910F91089581508B30C8F4EE
:104DC000FB01A82FBB27CD0182959295907F982754
:104DD000807F9827DC01A05EB64F80E190E021E063
:104DE0008030920719F40E94C4520895182E0E9430
:104DF000C452089581508B30C8F4FB01A82FBB2703
:104E0000CD0182959295907F9827807F9827DC012D
:104E1000A05EB64F80E190E021E08030920719F467
:104E20000E94B3520895182E0E94B3520895FC01B7
:104E3000DB018BE190E021E08030920719F40E94C1
:104E4000C45203C0182E0E94C45281E090E008951D
:104E5000FC01A0E1B0E082E190E021E08030920727
:104E600019F40E94C4520895182E0E94C452089545
:104E7000FC01A0E1B0E082E190E021E08030920707
:104E800019F40E94B3520895182E0E94B352089547
:104E9000FC01A0E3B0E084E290E021E080309207E2
:104EA00019F40E94C4520895182E0E94C452089505
:104EB000FC01A0E3B0E084E290E021E080309207C2
:104EC00019F40E94B3520895182E0E94B352089507
:104ED000FC01A0EDB2E088E190E021E08030920793
:104EE00019F40E94C4520895182E0E94C4520895C5
:104EF000FC01A0EDB2E088E190E021E08030920773
:104F000019F40E94B3520895182E0E94B3520895C6
:104F10000F93FC018081882319F488EE92E016C07B
:104F20008081813019F48EE293E010C0808182305C
:104F300019F484E793E00AC000E021E0AF0167E4E0
:104F400071E084E291E00E9469210DC0DC0186E4F9
:104F500090E021E08030920719F40E94C45203C00F
:104F6000182E0E94C4520F9108950F93CF93DF9390
:104F7000CDB7DEB721970FB6F894DEBF0FBECDBF19
:104F80008983882319F488EE92E018C089818130E2
:104F900019F48EE293E012C08981823019F484E71B
:104FA00093E00CC000E021E0AE014F5F5F4F60E690
:104FB00071E084E291E00E9469210EC0FB01DC01F6
:104FC00086E490E021E08030920719F40E94B35209
:104FD00003C0182E0E94B35221960FB6F894DEBF7C
:104FE0000FBECDBFDF91CF910F910895CF93DF9387
:104FF000CDB7DEB760970FB6F894DEBF0FBECDBF5A
:10500000FE013196A0E0B0E080E190E021E0803048
:10501000920719F40E94B35203C0182E0E94B35293
:105020008B858F3119F48FE190E008C08B85803239
:1050300019F480E290E002C08FE190E060960FB634
:10504000F894DEBF0FBECDBFDF91CF910895CFEDB5
:10505000D0E1DEBFCDBF0E9418410E94302B0E94DC
:10506000BE100E9402050E942A410E94C8350E947B
:105070008720FE013196A0E0B0E084E090E021E0DE
:105080008030920719F40E94B35203C0182E0E9478
:10509000B35244E050E068E371E0CE0101960E9413
:1050A0002D428823C1F18E010F5F1F4F80E2D8018E
:1050B0001D928A95E9F785E0E8E3F1E0D8010190D7
:1050C0000D928A95E1F71D821E821F82188619862D
:1050D0001A861B860E94D813F801A0E0B0E080E198
:1050E00090E021E08030920719F40E94C45203C07E
:1050F000182E0E94C452FE013196A0E0B0E084E078
:1051000090E021E08030920719F40E94C45203C05D
:10511000182E0E94C452FE013196A0E8B2E08AE047
:1051200090E021E08030920719F40E94B35203C04E
:10513000182E0E94B3524AE050E064E571E0CE01BF
:1051400001960E942D42882369F10E94F8130E9463
:10515000DB090E94F2430E94D705FE01319680E2EE
:10516000DF011D928A95E9F7A0E5BEE080E190E0BD
:1051700021E08030920719F40E94C45203C0182E17
:105180000E94C452E4E5F1E0A0E8B2E08AE090E0D9
:1051900021E08030920719F40E94C45203C0182EF7
:1051A0000E94C452FE013196A0E8B1E083E090E095
:1051B00021E08030920719F40E94B35203C0182EE8
:1051C0000E94B35243E050E06DE371E0CE010196DE
:1051D0000E942D42882391F00E94C720EDE3F1E068
:1051E000A0E8B1E083E090E021E08030920719F47C
:1051F0000E94C45203C0182E0E94C452FE01319670
:10520000A0E8B0E085E090E021E08030920719F45A
:105210000E94B35203C0182E0E94B35245E050E0E2
:1052200061E471E0CE0101960E942D42882309F4C9
:1052300075C0FE01319680E2DF011D928A95E9F783
:10524000ACEBB0E081E090E021E08030920719F40F
:105250000E94C45203C0182E0E94C452FE0131960F
:10526000A5E8B0E081E090E021E08030920719F4F9
:105270000E94C45203C0182E0E94C452FE013196EF
:10528000A6E8B0E082E090E021E08030920719F4D7
:105290000E94C45203C0182E0E94C452FE013196CF
:1052A000A8E8B0E082E190E021E08030920719F4B4
:1052B0000E94C45203C0182E0E94C452FE013196AF
:1052C000ACEAB0E080E190E021E08030920719F490
:1052D0000E94C45203C0182E0E94C452FE0131968F
:1052E000ADEBB0E082E190E021E08030920719F46C
:1052F0000E94C45203C0182E0E94C452E1E4F1E09F
:10530000A0E8B0E085E090E021E08030920719F459
:105310000E94C45203C0182E0E94C4520E94CC089E
:105320000E94422E0E94AF430E94E6140E941D3547
:1053300087E00E94504C78940E94743FA89580E0CA
:105340000E9430350E94D335FACF1F93162FA398B1
:10535000992787709070880F991F81640E9423415C
:10536000812F0E94234180E00E942341A39A992724
:105370001F9108950F931F93162F042FA398992719
:1053800087709070880F991F80640E942341812F3D
:105390000E942341802F0E942341A39A1F910F91C5
:1053A00008958091400990914109892BA1F581E0F0
:1053B00090E090934109809340094CE16AE080E0DD
:1053C0000E94BA2940E0642F842F0E94BA294FEF2F
:1053D00061E080E00E94BA2940E062E0842F0E94F0
:1053E000BA2940E063E0842F0E94BA2940E064E0DB
:1053F000842F0E94BA2940E065E0842F0E94BA29D8
:1054000040E06CE0842F0E94BA2940E06DE0842FD8
:105410000E94BA290895809140099091410901970D
:10542000A1F54CE16AE081E00E94BA2940E0642FD6
:1054300081E00E94BA294FEF61E0862F0E94BA29CD
:1054400040E062E081E00E94BA2940E063E081E050
:105450000E94BA2940E064E081E00E94BA2940E05D
:1054600065E081E00E94BA2940E06CE081E00E94A2
:10547000BA2940E06DE081E00E94BA2982E090E024
:10548000909341098093400908958091400990913B
:1054900041090297A1F54CE16AE082E00E94BA2935
:1054A00040E0642F82E00E94BA294FEF61E082E081
:1054B0000E94BA2940E062E0862F0E94BA2940E0AB
:1054C00063E082E00E94BA2940E064E082E00E944A
:1054D000BA2940E065E082E00E94BA2940E06CE031
:1054E00082E00E94BA2940E06DE082E00E94BA2981
:1054F00083E090E090934109809340090895809162
:105500004009909141090397A1F54CE16AE083E0DD
:105510000E94BA2940E0642F83E00E94BA294FEF2D
:1055200061E083E00E94BA2940E062E083E00E94EB
:10553000BA2940E063E0862F0E94BA2940E064E087
:1055400083E00E94BA2940E065E083E00E94BA2926
:1055500040E06CE083E00E94BA2940E06DE083E027
:105560000E94BA2984E090E0909341098093400919
:10557000089580914009909141090497A1F54CE16B
:105580006AE084E00E94BA294CEF60E084E00E9467
:10559000BA294FEF61E084E00E94BA2940E062E05E
:1055A00084E00E94BA2940E063E084E00E94BA29C6
:1055B00040E064E0862F0E94BA2940E065E084E084
:1055C0000E94BA2940E06CE084E00E94BA2940E0E1
:1055D0006DE084E00E94BA2985E090E09093410953
:1055E0008093400908958091400990914109059761
:1055F00091F54CE16AE085E00E94BA2940E0642F11
:1056000085E00E94BA2940EF61E085E00E94BA2956
:1056100040E062E085E00E94BA2940E063E085E076
:105620000E94BA2940E064E085E00E94BA2940E087
:1056300065E0862F0E94BA2940E06CE085E00E9478
:10564000BA2940E06DE085E00E94BA291092410934
:10565000109240090895109241091092400908954E
:105660009B9AA39A4CE16AE080E00E94BA2940E04C
:1056700064E1842F0E94BA2940E0642F842F0E94A5
:10568000BA294FEF61E080E00E94BA2940E062E071
:10569000842F0E94BA2940E063E0842F0E94BA2937
:1056A00040E064E0842F0E94BA2940E065E0842F46
:1056B0000E94BA2940E06CE0842F0E94BA2940E0A1
:1056C0006DE0842F0E94BA294CE16AE081E00E94DB
:1056D000BA2940E064E181E00E94BA2940E0642FE9
:1056E00081E00E94BA294FEF61E0862F0E94BA291B
:1056F00040E062E081E00E94BA2940E063E081E09E
:105700000E94BA2940E064E081E00E94BA2940E0AA
:1057100065E081E00E94BA2940E06CE081E00E94EF
:10572000BA2940E06DE081E00E94BA294CE16AE0CC
:1057300082E00E94BA2940E064E182E00E94BA2936
:1057400040E0642F82E00E94BA294FEF61E082E0DE
:105750000E94BA2940E062E0862F0E94BA2940E008
:1057600063E082E00E94BA2940E064E082E00E94A7
:10577000BA2940E065E082E00E94BA2940E06CE08E
:1057800082E00E94BA2940E06DE082E00E94BA29DE
:105790004CE16AE083E00E94BA2940E064E183E0E2
:1057A0000E94BA2940E0642F83E00E94BA294FEF9B
:1057B00061E083E00E94BA2940E062E083E00E9459
:1057C000BA2940E063E0862F0E94BA2940E064E0F5
:1057D00083E00E94BA2940E065E083E00E94BA2994
:1057E00040E06CE083E00E94BA2940E06DE083E095
:1057F0000E94BA294CE16AE084E00E94BA2940E0A4
:1058000064E184E00E94BA294CEF60E084E00E94E9
:10581000BA294FEF61E084E00E94BA2940E062E0DB
:1058200084E00E94BA2940E063E084E00E94BA2943
:1058300040E064E0862F0E94BA2940E065E084E001
:105840000E94BA2940E06CE084E00E94BA2940E05E
:105850006DE084E00E94BA294CE16AE085E00E9494
:10586000BA2940E064E185E00E94BA2940E065E1A0
:1058700085E00E94BA2940E0642F85E00E94BA29A1
:1058800040EF61E085E00E94BA2940E062E085E0F7
:105890000E94BA2940E063E085E00E94BA2940E016
:1058A00064E085E00E94BA2940E065E0862F0E940E
:1058B000BA2940E06CE085E00E94BA2940E06DE042
:1058C00085E00E94BA2908950F931F93CF93082F64
:1058D000C62F142F20E030E0613611F421E030E0D3
:1058E00080E090E0C13411F481E090E0822B932BB2
:1058F000892B91F060E0812F0E94A52921E030E002
:10590000002E02C0220F331F0A94E2F7482F422BC9
:1059100060E0812F0E94BA2920E030E0C23611F405
:1059200021E030E080E090E0C23411F481E090E0CA
:10593000822B932B892B89F061E0812F0E94A5296E
:1059400021E030E002C0220F331F0A95E2F7482F12
:10595000422B61E0812F0E94BA29CF911F910F91B4
:1059600008950F931F93CF93082FC62F142F20E075
:1059700030E0613611F421E030E080E090E0C134A5
:1059800011F481E090E0822B932B892BA1F060E051
:10599000812F0E94A52921E030E0002E02C0220FB5
:1059A000331F0A94E2F7922F9095482F492360E025
:1059B000812F0E94BA2920E030E0C23611F421E0A4
:1059C00030E080E090E0C23411F481E090E0822B7E
:1059D000932B892B99F061E0812F0E94A52921E06A
:1059E00030E002C0220F331F0A95E2F7922F909504
:1059F000482F492361E0812F0E94BA29CF911F913E
:105A00000F9108950F931F93CF93182FC62F042F34
:105A100020E030E0613611F421E030E080E090E0F9
:105A2000C13411F481E090E0822B932B892B29F073
:105A3000412F64E1802F0E94BA2920E030E0C23675
:105A400011F421E030E080E090E0C23411F481E014
:105A500090E0822B932B892B29F0412F65E1802F39
:105A60000E94BA29CF911F910F9108950F931F9310
:105A7000CF93082FC62F142F50E020E030E061367E
:105A800011F421E030E080E090E0C13411F481E0D5
:105A900090E0822B932B892B71F062E1812F0E9481
:105AA000A52921E030E0002E02C0220F331F0A9406
:105AB000E2F7582F522B20E030E0C23611F421E0FB
:105AC00030E080E090E0C23411F481E090E0822B7D
:105AD000932B892B69F063E1812F0E94A52921E096
:105AE00030E002C0220F331F0A95E2F7582F522BE5
:105AF000412F6C2F852F0E94022DCF911F910F9166
:105B000008950F931F93CF93082FC62F142F50E0A3
:105B100020E030E0613611F421E030E080E090E0F8
:105B2000C13411F481E090E0822B932B892B81F01A
:105B300062E1812F0E94A52921E030E0002E02C001
:105B4000220F331F0A94E2F7922F9095582F592372
:105B500020E030E0C23611F421E030E080E090E057
:105B6000C23411F481E090E0822B932B892B79F0E1
:105B700063E1812F0E94A52921E030E002C0220FBD
:105B8000331F0A95E2F7922F9095582F5923412FF2
:105B90006C2F852F0E94022DCF911F910F91089598
:105BA0001F93CF93C82F162F40E020E030E08136BE
:105BB00011F421E030E080E090E0C13411F481E0A4
:105BC00090E0822B932B892B29F062E1812F0E9498
:105BD000A529482F20E030E0C23611F421E030E062
:105BE00080E090E0C23411F481E090E0822B932BAE
:105BF000892B29F063E1812F0E94A529482F842F4A
:105C00009927CF911F9108950F931F93CF93182F2A
:105C1000C62F042F40E020E030E0613611F421E08F
:105C200030E080E090E0C13411F481E090E0822B1C
:105C3000932B892B29F062E1802F0E94A529482F00
:105C400020E030E0C23611F421E030E080E090E066
:105C5000C23411F481E090E0822B932B892B29F040
:105C600063E1802F0E94A529482F81E090E002C0C7
:105C7000880F991F1A95E2F784239927CF911F91D6
:105C80000F9108950E948D0C8FE999E09093360A48
:105C90008093350A1092370A10922E0A10922F0A1A
:105CA0008EE29AE00E949E0C8823D1F710922D0A72
:105CB00087EA99E09093420A8093410A1092430A3E
:105CC00010923A0A10923B0A8AE39AE00E949E0CD4
:105CD0008823D1F71092390A8FEA99E090934E0AFF
:105CE00080934D0A10924F0A1092460A1092470A6A
:105CF00086E49AE00E949E0C8823D1F71092450A10
:105D000087EB99E090935A0A8093590A10925B0AA4
:105D10001092520A1092530A82E59AE00E949E0C59
:105D20008823D1F71092510A8FE499E09093C70924
:105D30008093C6091092C8091092BF0982E080932F
:105D4000C0098FEB99E00E949E0C8823D1F787E56C
:105D500099E09093D2098093D1091092D3091092BF
:105D6000CA0982E08093CB098AEC99E00E949E0CDC
:105D70008823D1F78FE599E09093DD098093DC09C2
:105D80001092DE091092D50982E08093D60985ED44
:105D900099E00E949E0C8823D1F787E699E09093C2
:105DA000E8098093E7091092E9091092E00982E07E
:105DB0008093E10980EE99E00E949E0C8823D1F740
:105DC0008FE699E09093F3098093F2091092F40919
:105DD0001092EB0982E08093EC098BEE99E00E942F
:105DE0009E0C8823D1F787E799E09093FE09809372
:105DF000FD091092FF091092F60982E08093F709DD
:105E000086EF99E00E949E0C8823D1F78FE799E0F6
:105E10009093090A8093080A10920A0A1092010AC4
:105E200082E08093020A81E09AE00E949E0C88231F
:105E3000D1F787E899E09093140A8093130A10929F
:105E4000150A10920C0A82E080930D0A8CE09AE009
:105E50000E949E0C8823D1F78FE899E090931F0A47
:105E600080931E0A1092200A1092170A82E08093F3
:105E7000180A87E19AE00E949E0C8823D1F787E9EF
:105E800099E090932A0A8093290A10922B0A109283
:105E9000220A82E08093230A82E29AE00E949E0C0A
:105EA0008823D1F7089580912D0A8823E1F080910D
:105EB0002D0A813059F48DE29AE001960E949E0CE1
:105EC000882389F482E080932D0A0DC080912D0AE9
:105ED000823049F48DE29AE001960E94B00D882349
:105EE00011F480932D0A8091390A8823E1F0809182
:105EF000390A813059F489E39AE001960E949E0C98
:105F0000882389F482E08093390A0DC08091390A90
:105F1000823049F489E39AE001960E94B00D88230B
:105F200011F48093390A8091450A8823E1F0809129
:105F3000450A813059F485E49AE001960E949E0C4E
:105F4000882389F482E08093450A0DC08091450A38
:105F5000823049F485E49AE001960E94B00D8823CE
:105F600011F48093450A8091510A8823E1F08091D1
:105F7000510A813059F481E59AE001960E949E0C05
:105F8000882389F482E08093510A08958091510A10
:105F9000823049F481E59AE001960E94B00D882391
:105FA00011F48093510A0895CF93DF93EC018FEBA6
:105FB00099E00E94B00D882309F046C08091C10984
:105FC0009091C209AA27BB2788839983AA83BB83A0
:105FD000E091C609F091C70980818D83E091C609DF
:105FE000F091C70981818E83E091C609F091C709BC
:105FF00082818F83E091C609F091C70983818887E8
:10600000E091C609F091C70984818987E091C609AA
:10601000F091C70985818A87E091C609F091C70987
:1060200086818B87E091C609F091C70987818C87AB
:106030008091C5098C838FEB99E00E949E0C882388
:10604000D1F781E090E0BBC28AEC99E00E94B00DEC
:10605000882309F046C08091CC099091CD09AA27E8
:10606000BB2788839983AA83BB83E091D109F091F0
:10607000D20980818D83E091D109F091D20981818B
:106080008E83E091D109F091D20982818F83E091D2
:10609000D109F091D20983818887E091D109F091EB
:1060A000D20984818987E091D109F091D209858153
:1060B0008A87E091D109F091D20986818B87E0919E
:1060C000D109F091D20987818C878091D0098C8386
:1060D0008AEC99E00E949E0C8823D1F781E090E041
:1060E0006EC285ED99E00E94B00D882309F046C08C
:1060F0008091D7099091D809AA27BB2788839983D3
:10610000AA83BB83E091DC09F091DD0980818D8356
:10611000E091DC09F091DD0981818E83E091DC0959
:10612000F091DD0982818F83E091DC09F091DD0936
:1061300083818887E091DC09F091DD09848189877A
:10614000E091DC09F091DD0985818A87E091DC0925
:10615000F091DD0986818B87E091DC09F091DD0902
:1061600087818C878091DB098C8385ED99E00E9483
:106170009E0C8823D1F781E090E021C280EE99E067
:106180000E94B00D882309F046C08091E2099091E9
:10619000E309AA27BB2788839983AA83BB83E0915D
:1061A000E709F091E80980818D83E091E709F0919A
:1061B000E80981818E83E091E709F091E809828105
:1061C0008F83E091E709F091E80983818887E09166
:1061D000E709F091E80984818987E091E709F09166
:1061E000E80985818A87E091E709F091E8098681CD
:1061F0008B87E091E709F091E80987818C8780918E
:10620000E6098C8380EE99E00E949E0C8823D1F7EA
:1062100081E090E0D4C18BEE99E00E94B00D88231C
:1062200009F046C08091ED099091EE09AA27BB279D
:1062300088839983AA83BB83E091F209F091F309E3
:1062400080818D83E091F209F091F30981818E8341
:10625000E091F209F091F30982818F83E091F209D4
:10626000F091F30983818887E091F209F091F309B5
:1062700084818987E091F209F091F30985818A8709
:10628000E091F209F091F30986818B87E091F209A0
:10629000F091F30987818C878091F1098C838BEED3
:1062A00099E00E949E0C8823D1F781E090E087C19D
:1062B00086EF99E00E94B00D882309F046C08091D6
:1062C000F8099091F909AA27BB2788839983AA83A3
:1062D000BB83E091FD09F091FE0980818D83E091FF
:1062E000FD09F091FE0981818E83E091FD09F09115
:1062F000FE0982818F83E091FD09F091FE0983817F
:106300008887E091FD09F091FE0984818987E091F9
:10631000FD09F091FE0985818A87E091FD09F091E0
:10632000FE0986818B87E091FD09F091FE09878146
:106330008C878091FC098C8386EF99E00E949E0CEB
:106340008823D1F781E090E03AC181E09AE00E9491
:10635000B00D882309F046C08091030A9091040A89
:10636000AA27BB2788839983AA83BB83E091080A65
:10637000F091090A80818D83E091080AF091090A61
:1063800081818E83E091080AF091090A82818F83CE
:10639000E091080AF091090A83818887E091080A50
:1063A000F091090A84818987E091080AF091090A2D
:1063B00085818A87E091080AF091090A86818B8796
:1063C000E091080AF091090A87818C878091070A79
:1063D0008C8381E09AE00E949E0C8823D1F781E0B3
:1063E00090E0EDC08CE09AE00E94B00D882309F0A7
:1063F00046C080910E0A90910F0AAA27BB27888376
:106400009983AA83BB83E091130AF091140A8081D7
:106410008D83E091130AF091140A81818E83E091BB
:10642000130AF091140A82818F83E091130AF0918C
:10643000140A83818887E091130AF091140A8481F9
:106440008987E091130AF091140A85818A87E09187
:10645000130AF091140A86818B87E091130AF09158
:10646000140A87818C878091120A8C838CE09AE0D1
:106470000E949E0C8823D1F781E090E0A0C087E1C4
:106480009AE00E94B00D882309F046C08091190A55
:1064900090911A0AAA27BB2788839983AA83BB8372
:1064A000E0911E0AF0911F0A80818D83E0911E0AFF
:1064B000F0911F0A81818E83E0911E0AF0911F0ADC
:1064C00082818F83E0911E0AF0911F0A8381888761
:1064D000E0911E0AF0911F0A84818987E0911E0ACB
:1064E000F0911F0A85818A87E0911E0AF0911F0AA8
:1064F00086818B87E0911E0AF0911F0A87818C8725
:1065000080911D0A8C8387E19AE00E949E0C88236B
:10651000D1F781E090E053C082E29AE00E94B00D92
:10652000882309F046C08091240A9091250AAA2761
:10653000BB2788839983AA83BB83E091290AF091C2
:106540002A0A80818D83E091290AF0912A0A8181AB
:106550008E83E091290AF0912A0A82818F83E0914B
:10656000290AF0912A0A83818887E091290AF0910B
:106570002A0A84818987E091290AF0912A0A858173
:106580008A87E091290AF0912A0A86818B87E09117
:10659000290AF0912A0A87818C878091280A8C83A6
:1065A00082E29AE00E949E0C8823D1F781E090E07D
:1065B00006C0188219821A821B8280E090E0DF9167
:1065C000CF910895CF93DF93DC0180912D0A88232A
:1065D00039F48DE29AE090935E0A80935D0A21C0BF
:1065E0008091390A882339F489E39AE090935E0A0E
:1065F00080935D0A16C08091450A882339F485E4AA
:106600009AE090935E0A80935D0A0BC08091510AD4
:10661000882309F072C081E59AE090935E0A809326
:106620005D0AE0915D0AF0915E0A0084F185E02D3B
:10663000ED018D818083E0915D0AF0915E0A008416
:10664000F185E02D8E818183E0915D0AF0915E0AF3
:106650000084F185E02D8F818283E0915D0AF091C5
:106660005E0A0084F185E02D88858383E0915D0AD0
:10667000F0915E0A0084F185E02D89858483E091A4
:106680005D0AF0915E0A0084F185E02D8A8585839C
:10669000E0915D0AF0915E0A0084F185E02D8B8522
:1066A0008683E0915D0AF0915E0A0084F185E02D19
:1066B0008C858783E0915D0AF0915E0A8C818783E7
:1066C000E0915D0AF0915E0A8D919C9194838383A1
:1066D000E0915D0AF0915E0A1286E0915D0AF09108
:1066E0005E0A1182E0915D0AF0915E0A1282E091E9
:1066F0005D0AF0915E0A81E08083DF91CF91089579
:1067000082E499E00E94D42F882361F182E499E029
:106710000E94B90A82E499E00E94D42F882311F1E3
:1067200082E499E00E94B90A82E499E00E94D42FA1
:106730008823C1F082E499E00E94B90A82E499E0DA
:106740000E94D42F882371F082E499E00E94B90A54
:1067500082E499E00E94D42F882321F082E499E01A
:106760000E94B90A0895FF920F931F93CF93DF936E
:10677000CDB7DEB760970FB6F894DEBF0FBECDBFC2
:1067800020E0822F9927880F991F880F991F8C016D
:10679000015A154FF8011082F22EF394BE016F5F7B
:1067A0007F4F8F2D0E94FA268889F80182831382F9
:1067B00011822F2D2B3028F360960FB6F894DEBF90
:1067C0000FBECDBFDF91CF911F910F91FF90089524
:1067D000FC0180819927009719F0019731F0089505
:1067E00082E0838381E0808308958381882389F414
:1067F0008281882329F481E0818382E08083089567
:106800008181813011F4118202C081E0818382E0B4
:1068100080830895FC0180819927813091059CF047
:10682000833091051CF0039731F0089582E0838353
:1068300083E0808308958381882329F48083828183
:10684000882309F48183089520E0822F9927880FF7
:10685000991F880F991FFC01E15AF54F8381882306
:1068600011F0815083832F5F2B3078F3EFE5FAE04E
:10687000309B04C0CF010E94E83303C0CF010E94C7
:106880000A34E3E6FAE0319904C0CF010E94E8330C
:1068900003C0CF010E940A34E7E6FAE0329904C04F
:1068A000CF010E94E83303C0CF010E940A34EBE617
:1068B000FAE0499904C0CF010E94E83303C0CF0138
:1068C0000E940A34EFE6FAE0349904C0CF010E9436
:1068D000E83303C0CF010E940A34E3E7FAE03599B8
:1068E00004C0CF010E94E83303C0CF010E940A34E4
:1068F000E7E7FAE0369904C0CF010E94E83303C00D
:10690000CF010E940A34EBE7FAE0379904C0CF01C7
:106910000E94E83303C0CF010E940A34EFE7FAE097
:10692000339904C0CF010E94E83303C0CF010E9415
:106930000A34E3E8FAE04A9904C0CF010E94E83340
:1069400003C0CF010E940A34E7E8FAE04B9904C083
:10695000CF010E94E8330895CF010E940A340895C0
:106960009927853C910509F43FC0863C9105A4F424
:10697000823C910569F1833C91053CF4803C910592
:10698000F9F0813C910501F147C0833C9105C1F1CB
:10699000843C910529F140C0813D9105E9F0823D9B
:1069A00091053CF4863C910519F1873C910521F154
:1069B00033C0823D910541F1833D910549F12CC0E1
:1069C0008091600A992708958091640A9927089513
:1069D0008091680A9927089580916C0A99270895F3
:1069E0008091700A992708958091740A99270895D3
:1069F0008091780A9927089580917C0A99270895B3
:106A00008091800A992708958091840A9927089592
:106A10008091880A992708958EEF90E0089510924A
:106A2000B60087E08093B0001092B2008EE48093AD
:106A3000B30082E08093700008950E940F35109299
:106A40008D0A10928E0A10928F0A1092940A109258
:106A5000950A0E94B3330E9480050E948122089506
:106A6000CF93C82F80918B0A882311F010928B0A44
:106A7000A8950E948033C23011F00E94532FC2307B
:106A800009F463C080918C0A8823C9F180918C0A33
:106A9000815080938C0A80918D0A8F5F80938D0A3C
:106AA000823040F010928D0A0E9424340E943E0EE3
:106AB0000E94540680918E0A8F5F80938E0A8430E4
:106AC00040F010928E0A0E94450E0E9426440E94B9
:106AD000354180918F0A8F5F80938F0A843178F0DF
:106AE00010928F0A8091940A8F5F8093940A0E947B
:106AF0009E0E0E94750AC13011F00E94A00A80917A
:106B0000940A8A3010F11092940A8091900A909120
:106B1000910AA091920AB091930A0196A11DB11D0C
:106B20008093900A9093910AA093920AB093930A4B
:106B30000E9489238091950A8F5F8093950A8C33F8
:106B400020F01092950A0E944823CF9108958091D9
:106B5000900A9091910AA091920AB091930ABC0177
:106B6000CD0108951F920F920FB60F9211248F93AB
:106B70001092B20081E080938B0A80918C0A8F5F23
:106B800080938C0A8F910F900FBE0F901F901895D5
:106B90000E94CB3F0E94804160E076E980E090E077
:106BA0000E949B41089504C00E9411400E946F40C2
:106BB0000E94FB3F8823C1F70895FC0190E06150DB
:106BC0006F3F21F0819198276150E0F7892F992735
:106BD00008950F931F938C01FC0181818150682FD0
:106BE000C80101960E94DD35F801808381819927D3
:106BF000BC01C8010E942C401F910F910895AF92D3
:106C0000BF92CF92DF92EF92FF920F931F93CF9399
:106C1000DF93CDB7DEB7C45ED0400FB6F894DEBFC9
:106C20000FBECDBF6C01FC0181818150682FC60170
:106C300001960E94DD35D6019C91981711F00C94B5
:106C4000593FF6018281882309F0FBC0838199278F
:106C50008135910509F449C0823591053CF48033B2
:106C6000910589F08035910561F1EBC0833591057F
:106C700009F491C0833591050CF47BC084359105EE
:106C800009F4B5C0DEC08E01025D1F4F80E5D8015A
:106C90001D928A95E9F785E18FA718AA80E889AB4C
:106CA000F60184818AAB992796012B5F3F4FAC0197
:106CB000B901CE01C3960E94C751C8010E94E935AF
:106CC000C0C08E01025D1F4F80E5D8011D928A95DC
:106CD000E9F785E08FA718AA80EA89AB0E940F2107
:106CE0008AABC8010E94E935ACC0F601B4800F2E12
:106CF000FEE2EF2EFF24F02DEC0EFD1E80E5D70105
:106D00001D928A95E9F789E18FA718AA81EA89ABD4
:106D10008E0102581F4FB8018B2D0E943921BAAA4B
:106D20008CE0FE01F396D8010D9001928A95E1F76F
:106D3000F80184859585FE01FF9691838083F80193
:106D40008685FE01EF5BFF4F8083F8018785FE019A
:106D5000EE5BFF4F80839927AC01BE0162577F4FE6
:106D6000CE018D5B9F4F0E94C751C7010E94E9353C
:106D700068C00E94C720FE01BE9680E5DF011D921B
:106D80008A95E9F784E08FA718AA82EA89ABCF0138
:106D90000E94E93556C0F601458156818481FE0185
:106DA000EC51FF4F8083813108F04BC080E5FE013C
:106DB000BE9611928A95E9F787E18FA718AA83EA10
:106DC00089AB5CAB4BABFE01EC51FF4F80818AABD2
:106DD000FE01F5969927DA01019724F00E94AB5243
:106DE0000192FACFCE018E960E94E9352AC0F601B3
:106DF000458156818481FE01EC51FF4F80838131B2
:106E000000F5F60137969927DA01019724F00190F1
:106E10000E94B852FACFDE019E9680E5FD011192E4
:106E20008A95E9F787E08FA718AA84EA89AB5CAB5B
:106E30004BABFE01EC51FF4F80818AABCD010E942C
:106E4000E935F6018281813011F00C94623F838133
:106E50009927AA27BB27FC013197E536F10510F0E9
:106E60000C944B3FE65BFF4FEE0FFF1F0590F49134
:106E7000E02D09940E941F1FF601B4808B2D8150D4
:106E8000823210F00C94623F40E09E01275F3F4F3A
:106E9000842F9927D901A80FB91FF601E80FF91F10
:106EA00082858C934F5F4F3098F3F60185818983FB
:106EB00086818A8387818B83838D948D9E838D8346
:106EC000858D8F838085888781858C83818D888F50
:106ED000828D898F6B2DCE0101960E9446266B2DE7
:106EE000CE0101960E9480151EA685E08FA711E0B5
:106EF00018AB81E889AB1AAACE018E960E94E935BB
:106F0000812F0E943035DEC7F601B4808B2D815071
:106F1000823208F046C06B2DCE0101960E948B266E
:106F20008EE18FA781E088AB82E889ABBAAA89811C
:106F30008BAB8A818CAB8B818DAB8C818FAB8D8140
:106F40009E81FE01E75BFF4F918380838F81FE016D
:106F5000E55BFF4F808340E0BE016F5F7F4F9E0186
:106F6000275F3F4F842F9927DC01A60FB71FF90138
:106F7000E80FF91F8081FD0187AB4F5F4F3090F321
:106F800088858EAB888DFE01E95BFF4F8083898DFC
:106F9000FE01E85BFF4F8083CE018E960E94E935AB
:106FA00091C7FFEFBF1609F08DC7FE01EC51FF4FEF
:106FB0001082FE01EC51FF4F8081982F823208F041
:106FC00081C70F2EF4EEEF2EFF24F02DEC0EFD1EE8
:106FD0006E010894C11CD11C8E01075F1F4F892FC1
:106FE0008F5F682FCE0101960E948B268EE18FA7BE
:106FF00081E088AB82E889ABD7018C918F5F8AAB47
:1070000089818BAB8A818CAB8B818DAB8C818FAB73
:107010008D819E81FE01E75BFF4F918380838F818D
:10702000FE01E55BFF4F808340E0842F9927DC0160
:10703000AC0DBD1DF801E80FF91F8081FD0187AB84
:107040004F5F4F3090F388858EAB888DFE01E95BF2
:10705000FF4F8083898DFE01E85BFF4F8083CE0167
:107060008E960E94E93581E00E943035D7018C91DF
:107070008F5F8C93982F823208F4B1CF23C70E9480
:107080001F1FF601B480AE0142585F4F96012B5F7F
:107090003F4F8FE0DA01F90101900D928A95E1F7F7
:1070A000F6018489FA018787BA018B2D0E94DD26BB
:1070B00081E088AB83E889ABBAAA85E08FA7CE01CF
:1070C0008E960E94E935FEC6F601B4808B2D815064
:1070D0008A3008F581E088AB84E889ABBAAA8E01D2
:1070E00002581F4FB8018B2D0E94FA268FE0FE0137
:1070F000F396D8010D9001928A95E1F7F801878502
:10710000FE01EE5BFF4F808385E18FA7CE018E9657
:107110000E94E935D7C6FFEFBF1609F0D3C6FE01BE
:10712000EC51FF4F1082FE01EC51FF4F8081982FF0
:107130008B3008F0C7C6BB24B3948E0102581F4F92
:107140000F2EFFE0AF2EF02D0F2EF2E4EF2EFF24D6
:10715000F02DEC0EFD1E0F2EF4EECF2EDD24F02DC3
:10716000CC0EDD1EB8AA84E889AB892F8F5F8AAB6D
:10717000B8010E94FA26FE01F396D8012A2D0D903F
:1071800001922A95E1F7F8018785D7018C9385E173
:107190008FA7CE018E960E94E9358B2D0E94303547
:1071A000F60180818F5F8083982F8B30D8F28AC65A
:1071B0000E941F1F0E94BE10A8950E94F813A89558
:1071C0000E94E614A8950E94DB09A8950E94F2434C
:1071D000A8950E94D705A8950E94EE2281E088AB71
:1071E00086E889AB84E08FA7CE018E960E94E935B0
:1071F00069C684E18FA781E088AB87E889AB8DE021
:10720000A7E4B1E0FE01F2960D9001928A95E1F7B4
:107210000E94A7359B01AC01AA27BB278FAFBB27D4
:10722000A52F942F832FFE01E05CFF4F8083FE018A
:10723000EF5BFF4F2083CE018E960E94E93542C658
:107240000C9400003FC6C60104960E94D42481E03D
:1072500088AB89E889AB84E08FA7CE018E960E9427
:10726000E93530C681E088AB8AE889AB8CE08FA72E
:10727000CE01C2960E94E424CE018E960E94E9358A
:1072800021C6CE0189960E949D1C81E088AB81EACF
:1072900089AB89A58AAB8AA58BAB8BA58CAB8CA55A
:1072A0008DAB8DA58EAB89E08FA7CE018E960E9407
:1072B000E93508C6F601B480F1E2FB15F8F0BE012D
:1072C0006C5D7F4F8B2D0E94551D81E088AB82EA5B
:1072D00089ABBAAA8DA18CAB8EA18FAB8CA18BABE5
:1072E0008FA198A5892F99278DAB8FA18EAB8AE0AE
:1072F0008FA7CE018E960E94E935E4C52FEFB21616
:1073000009F0E0C5FE01EC51FF4F1082FE01EC5187
:10731000FF4F8081982F823208F0D4C5FF24F39468
:107320008F01BE016C5D7F4F892F8F5F0E94551DBD
:10733000F8AA82EA89ABD8018C918F5F8AAB8DA1C4
:107340008CAB8EA18FAB8CA18BAB8FA198A5892F15
:1073500099278DAB8FA18EAB8AE08FA7CE018E9639
:107360000E94E9358F2D0E943035F80180818F5FB2
:107370008083982F8232A8F2A5C5CE014C960E9438
:107380001B1E8AE08FA781E088AB80EA89AB8AA1C7
:107390008AAB88A18BAB8C8D9D8D892F99278CAB67
:1073A0008C8D8DAB8F8D8EAB8E8D8FABCE018E96EF
:1073B0000E94E93587C5F601648180E00E940417C8
:1073C00084E08FA781E088AB83EA89ABCE018E96FB
:1073D0000E94E93577C5DE01A253BF4FF6018481D3
:1073E0008C938581FD018183F6018681FD01828375
:1073F000F6018781FD018383F6018085FD01848389
:10740000F6018185FD018583F6018285FD01868374
:10741000F6018385FD018783CD010E94071784E073
:107420008FA781E088AB84EA89ABCE018E960E945B
:10743000E93548C5FE01E258FF4FA0E0B0E080E129
:1074400090E021E08030920719F40E94B35203C00B
:10745000182E0E94B352F60184819581A681B781CE
:10746000FE01EE57FF4F80839183A283B383DE0139
:10747000A258BF4FF6018085FD018087F601818506
:10748000FD018187F6018285FD018287A0E0B0E0E1
:1074900080E190E021E08030920719F40E94C4520C
:1074A00003C0182E0E94C45284E08FA781E088ABED
:1074B00080EC89ABCE018E960E94E93503C5FE01B2
:1074C000E258FF4FA0E0B0E080E190E021E08030A2
:1074D000920719F40E94B35203C0182E0E94B352AF
:1074E0008BE08FA781E088AB81EC89ABFE01EE5782
:1074F000FF4F80819181A281B3818AAB9BABACAB02
:10750000BDABFE01E258FF4F80858EAB81858FAB0E
:10751000828588AFCE018E960E94E935D3C48AE376
:107520008FA781E088AB80ED89ABFE01F296A8E8D9
:10753000B0E082E190E021E08030920719F40E94EF
:10754000B35203C0182E0E94B352FE01EC5BFF4FF2
:10755000AAE9B0E082E190E021E08030920719F4DE
:107560000E94B35203C0182E0E94B352FE01EA5A81
:10757000FF4FADEBB0E082E190E021E08030920778
:1075800019F40E94B35203C0182E0E94B352CE01C8
:107590008E960E94E93596C484E18FA781E088AB7E
:1075A0008EED89ABFE01F296ACEAB0E080E190E0AE
:1075B00021E08030920719F40E94B35203C0182EC4
:1075C0000E94B352CE018E960E94E9357BC40E9480
:1075D000EE2284E08FA781E088AB81ED89ABCE01FC
:1075E0008E960E94E9356EC488E08FA781E088AB53
:1075F0008FED89AB0E9480238CAB0E9484239BABD0
:107600008AABFE01EC51FF4FACEBB0E081E090E0C3
:1076100021E08030920719F40E94B35203C0182E63
:107620000E94B352FE01EC51FF4F80818DABCE0121
:107630008E960E94E93546C4FE01E258FF4F80E570
:10764000DF011D928A95E9F7ACEBB0E081E090E0B4
:1076500021E08030920719F40E94C45203C0182E12
:107660000E94C452FE01E258FF4FA5E8B0E081E05D
:1076700090E021E08030920719F40E94C45203C0C8
:10768000182E0E94C452FE01E258FF4FA6E8B0E057
:1076900082E090E021E08030920719F40E94C45209
:1076A00003C0182E0E94C45284E08FA781E088ABEB
:1076B00080EE89ABCE018E960E94E93503C4DE01CF
:1076C000AA52BF4FF60184818C938581FD0181838D
:1076D000D60116968CE0FE01E852FF4F0D90019204
:1076E0008A95E1F7FE01EC51FF4F1082FE01EC514B
:1076F000FF4F8081982F8C30A0F49E012A523F4F7B
:10770000DF01F901E90FF11D8281882321F08F3F0C
:1077100011F0815082838C918F5F8C93982F8C30E5
:1077200080F3CE018A529F4F0E94862484E08FA767
:1077300081E088AB87EA89ABCE018E960E94E9355D
:10774000C1C38E010A521F4FC8010E94A42482E1C6
:107750008FA781E088AB88EA89ABD8018C918AAB8E
:10776000F80181818BABFE01EC51FF4F1082FE01CD
:10777000EC51FF4F8081982F8C3080F49801DF010D
:10778000F901E90FF11D82818F3F11F08F5F828334
:107790008C918F5F8C93982F8C3090F38CE0DE016E
:1077A000A852BF4FFE01F4960D9001928A95E1F721
:1077B000CE018E960E94E93585C3F6018481FE01D3
:1077C000E258FF4F8083D601159680E1FE01E15813
:1077D000FF4F0D9001928A95E1F7FE01EC51FF4FAA
:1077E0001082FE01EC51FF4F8081982F8031A0F470
:1077F0009E0122583F4FDF01F901E90FF11D818100
:10780000882321F08F3F11F0815081838C918F5F0D
:107810008C93982F803180F3CE0182589F4F0E9425
:10782000B42484E08FA781E088AB89EA89ABCE01DC
:107830008E960E94E93546C38E0102581F4FC8013B
:107840000E94C42485E18FA781E088AB8AEA89ABD6
:10785000D8018C918AABFE01EC51FF4F1082FE01E2
:10786000EC51FF4F8081982F803180F49801DF0127
:10787000F901E90FF11D81818F3F11F08F5F818345
:107880008C918F5F8C93982F803190F380E1DE0193
:10789000A158BF4FFE01F3960D9001928A95E1F732
:1078A000CE018E960E94E9350DC3F601B480858124
:1078B0009927982F88272681820F911DBC018B2D37
:1078C0000E94881E85E08FA781E088AB82EC89AB9F
:1078D000BAAACE018E960E94E935F4C2F601B480B0
:1078E0008CE08FA781E088AB83EC89ABBAAA8B2DA3
:1078F0000E94461E8BAB8B2D0E94621E892F9927FA
:107900008CAB8B2D0E94621E8DAB8B2D0E94B11E05
:10791000892F99278EAB8B2D0E94B11E8FAB8B2D9B
:107920000E94C91E892F992788AF8B2D0E94C91EDE
:1079300089AFCE018E960E94E935C4C240E0F601BF
:10794000848181FD41E0F601848182FD4260842FC3
:107950000E94E11EB7C20E94E41E84E08FA718AA0D
:1079600085EC89ABCE018E960E94E935ABC2F6015B
:10797000B4809E0122583F4F8581D9018C93868126
:107980009781F90192838183F60180859185F901C0
:1079900094838383F6018685F9018187F6018785C3
:1079A000F9018287F60182859385F90196838583A3
:1079B000F60184859585F90190878783F601808992
:1079C000F9018387F6018189F9018487F6018289AB
:1079D000F9018587F6018389F9018687D6015496D6
:1079E0008FE0FE01E357FF4F0D9001928A95E1F77A
:1079F000F60183A1F901868FF60184A1F901878F31
:107A0000F60185A1F90180A3F60186A1F90181A300
:107A100015E0D6019796FE01E056FF4F812F0D909D
:107A200001928A95E1F7F60184A595A5A6A5B7A5CB
:107A3000F90187A390A7A1A7B2A7F60180A9F90130
:107A400083A7B9018B2D0E94662581E088AB82ED6A
:107A500089AB1FA7BAAACE018E960E94E93532C221
:107A6000F601B4808E0102581F4FB8018B2D0E9481
:107A70009E2581E088AB83ED89AB81E38FA7BAAA0D
:107A8000D8018C918BABF801818192819DAB8CAB3D
:107A9000838194819FAB8EAB81858CAF82858DAFC6
:107AA0008581968199AF88AF878190859BAF8AAF9A
:107AB00083858EAF84858FAF8585FE01E05CFF4FA7
:107AC0008083F8018685FE01EF5BFF4F80838FE0A6
:107AD000DE01A357BF4FFE01EE5BFF4F0D900192F9
:107AE0008A95E1F7F801868DFE01EF5AFF4F8083FA
:107AF000F801878DFE01EE5AFF4F8083F80180A1C7
:107B0000FE01ED5AFF4F8083F80181A1FE01EC5A7E
:107B1000FF4F808385E0DE01A056BF4FFE01EB5A88
:107B2000FF4F0D9001928A95E1F7F80187A190A58A
:107B3000A1A5B2A5FE01E65AFF4F80839183A283DF
:107B4000B383F80183A5FE01E25AFF4F8083CE0183
:107B50008E960E94E935B6C1F601B480AE01425856
:107B60005F4F828DDA018C93838DFA018183F60158
:107B7000848DFA018283F6018681FA018383F601FE
:107B80008781FA018483F6018085FA018583F601F5
:107B90008185FA018683F6018285FA018783F601E1
:107BA000858DFA01878BC6010B962FE0FE01EA57FF
:107BB000FF4FDC010D9001922A95E1F7BA018B2D60
:107BC0000E94D62581E088AB84ED89AB85E08FA744
:107BD000BAAACE018E960E94E93574C1F601B4802E
:107BE0008E0102581F4FB8018B2D0E940E2681E096
:107BF00088AB85ED89AB8FE18FA7BAAAD8018C91AC
:107C0000FE01E85BFF4F8083F8018181FE01E75BA5
:107C1000FF4F8083F8018281FE01E65BFF4F808386
:107C2000F80183818CAB84818DAB85818EAB86819D
:107C30008FAB878188AF8789FE01E55BFF4F80832B
:107C40008FE0DE01AA57BF4FFE01F9960D90019219
:107C50008A95E1F7CE018E960E94E93533C1F6018F
:107C60003496A0E9B7E080E190E021E0803092070F
:107C700019F40E94C45203C0182E0E94C45281E01D
:107C800088AB83EE89AB84E08FA7CE018E960E94ED
:107C9000E93518C181E088AB84EE89AB84E18FA718
:107CA000FE01F296A0E9B7E080E190E021E08030AB
:107CB000920719F40E94B35203C0182E0E94B352C7
:107CC000CE018E960E94E935FDC0F601B480C60152
:107CD0000596BC018B2D0E94F42481E088AB88EDD1
:107CE00089AB85E08FA7BAAACE018E960E94E935AE
:107CF000E9C0F601B48081E088AB89ED89AB8DE104
:107D00008FA7BAAABE016D5C7F4F8B2D0E942D25D7
:107D1000CE018E960E94E935D5C0C60105960E9417
:107D2000682781E088AB86ED89AB85E08FA7CE011F
:107D30008E960E94E935C6C081E088AB87ED89AB9D
:107D40008DE18FA7CE01C3960E947827CE018E9633
:107D50000E94E935B7C0F601B480C60104960E94BE
:107D6000882781E088AB8AED89AB85E08FA7BAAA26
:107D7000CE018E960E94E935A5C0F601B48081E05F
:107D800088AB8BED89AB8AE48FA7BE016E5C7F4F19
:107D90008B2D0E94B527CE018E960E94E93592C0A8
:107DA000F601B4808B2D0E94440A81E088AB8CEDF3
:107DB00089ABBAAA85E08FA7CE018E960E94E935DD
:107DC00081C0F6014481558181E088AB8DED89AB9E
:107DD00086E18FA75BAB4AABFE01EC51FF4F1082EF
:107DE000FE01EC51FF4F8081982F8031C8F48E0145
:107DF0000F5F1F4FBF01892F99279C01200F311F53
:107E0000840F951FAA27BB27ABBFFC018791F901FF
:107E100083ABDB018C918F5F8C93982F803158F36B
:107E2000CE018E960E94E9354DC0F6013496A0E54C
:107E3000BEE080E190E021E08030920719F40E94DA
:107E4000C45203C0182E0E94C45281E088AB81EE58
:107E500089AB84E08FA7CE018E960E94E93532C0AF
:107E600081E088AB82EE89AB84E18FA7FE01F296B8
:107E7000A0E5BEE080E190E021E08030920719F4B7
:107E80000E94B35203C0182E0E94B352CE018E96A8
:107E90000E94E93517C081E088AB80E889AB85E0B6
:107EA0008FA7F60183818AABCE018E960E94E935B9
:107EB00009C085E08FA718AA81E089ABCE018E9614
:107EC0000E94E935CC51DF4F0FB6F894DEBF0FBEEC
:107ED000CDBFDF91CF911F910F91FF90EF90DF9079
:107EE000CF90BF90AF900895CF93DF93CDB7DEB71B
:107EF0002A970FB6F894DEBF0FBECDBF81E08B830B
:107F000088E88C8384E08A83CE0101960E94E9355B
:107F10002A960FB6F894DEBF0FBECDBFDF91CF918A
:107F200008950F931F93CF93DF93CDB7DEB7C0555E
:107F3000D0400FB6F894DEBF0FBECDBF8A0121E05E
:107F40002B832DE52C839E838D836F8320E0261762
:107F500080F4AE01485F5F4F822F9927DA01A80FA6
:107F6000B91FF801E80FF91F80818C932F5F261746
:107F700098F38FE08A83CE0101960E94E935C05BB9
:107F8000DF4F0FB6F894DEBF0FBECDBFDF91CF91AC
:107F90001F910F91089548EC50E060E070E087E990
:107FA0009AE00E94D45110925F0B1092600B1092D5
:107FB000960A0895382F2091600B87E99AE0FC011A
:107FC000E20FF11D30838091600B8F5F8093600B17
:107FD0008091960A8F5F8093960A8091960A883CDA
:107FE00018F00E94CB3F08958091600B883C10F000
:107FF0001092600B08959091600B80915F0B981721
:1080000038F08091600B90915F0B891B9927089540
:108010009091600B80915F0B981B892F8853992753
:10802000089520915F0B87E99AE0FC01E20FF11DB2
:10803000E08180915F0B8F5F80935F0B8091960A48
:1080400081508093960A80915F0B883C10F01092CB
:108050005F0B8E2F992708950F931F93CF93DF9374
:108060008C01EB0180EC0E94C14121978FEFCF3F43
:10807000D80769F1CE0165E070E00E942452892B97
:1080800019F081E00E943035F80180819927803C09
:10809000910521F08B3D910541F00EC08BED0E94C2
:1080A000C1418CED0E94C1410BC08BED0E94C141CA
:1080B0008DED0E94C14104C0F80180810E94C14140
:1080C0000F5F1F4F2197FFEFCF3FDF0799F680EC3F
:1080D0000E94C141DF91CF911F910F9108950F939D
:1080E0001F93382F8091610B9927009719F0019702
:1080F000C1F059C0303C09F056C01092620B20917B
:10810000620B84E69BE0FC01E20FF11D30832F5FE0
:108110002093620B81E08093610B84E68093630B74
:1081200042C0303C99F58091620B8230F0F0809132
:10813000620B04E61BE0F801E80FF11D30838F5F4E
:108140008093620B82E08093610B1092630BA80115
:108150006091620BC8010E94DE40C8010E94FF3599
:108160001092610B1092620B1EC01092620B209154
:10817000620B84E69BE0FC01E20FF11D30832F5F70
:108180002093620B84E68093630B0DC02091620BF9
:1081900084E69BE0FC01E20FF11D30838091620BCD
:1081A0008F5F8093620B8091620B893620F0109272
:1081B000610B1092620B1F910F910895FC01DA017F
:1081C00061506F3FF1F02081822F9927803C91050B
:1081D00021F08B3D910519F010C0319610C03196F9
:1081E0002081822F99278C3D910521F08D3D9105AD
:1081F00019F003C020EC01C02BED2D933196615096
:1082000010F708958091630B882389F08091630BA8
:1082100081508093630B9091630B992341F480917B
:10822000610B813021F49093620B9093610B089560
:1082300085B1807F85B984B1876084B981E58CBDC3
:1082400081E08DBD08958EBD0DB407FEFDCF8EB5C6
:10825000992708950E947E419C9AA4988FE080936C
:10826000CE0BA4986A9862980895CF93DF93CDB708
:10827000DEB728970FB6F894DEBF0FBECDBFA49B24
:1082800011C062990DC08091CD0B853018F0A49873
:108290000E94FA158091CD0B8F5F8093CD0B02C0A9
:1082A0001092CD0BCE0101960E941B1E29813A81AE
:1082B00081E590E0289FA001299F500D389F500D27
:1082C0001124CA01880F892F881F990B91950E944C
:1082D0007F418D81882319F48F81882311F0A49A1E
:1082E00001C0A49828960FB6F894DEBF0FBECDBF8C
:1082F000DF91CF9108958093CE0B0895089508954E
:108300001092D00B1092CF0B86E08093C20088EDC4
:108310008093C10060E875E280E090E00E949B419C
:1083200081E080931D0E10921E0E08959093D00B45
:108330008093CF0B08959B01AC01DC01CB016894C5
:1083400012F8880F991FAA1FBB1F1694D1F78050EF
:108350009C4DAB40BF4F689413F8220F331F441F4E
:10836000551F1694D1F7BC01CD010E943752DA0196
:10837000C9010197292F33272093C5008093C4009A
:108380000895982F80911D0E8823E1F310921D0E01
:108390009093C60008950F931F93CF93DF938C01A2
:1083A000EB0121978FEFCF3FD80751F0F801819172
:1083B0008F010E94C1412197FFEFCF3FDF07B1F747
:1083C00081E090E0DF91CF911F910F9108951F926E
:1083D0000F920FB60F9211248F9381E080931D0EA0
:1083E0008F910F900FBE0F901F9018951F920F92B4
:1083F0000FB60F9211242F933F934F935F936F9378
:108400007F938F939F93AF93BF93EF93FF9380914D
:10841000C6000E94DA3FFF91EF91BF91AF919F910B
:108420008F917F916F915F914F913F912F910F901D
:108430000FBE0F901F901895DC01FB01415050407A
:108440008FEF4F3F580741F081918D93415050403D
:108450008FEF4F3F5807C1F70895DC01FB014150F2
:1084600050408FEF4F3F580769F091918D918917D8
:1084700019F081E090E00895415050408FEF4F3F58
:10848000580799F780E090E00895CF93DF93DC01DF
:10849000FB0160E0462F91E0562F8081803231F45D
:1084A000692F9F5F319680818032D1F3808188234C
:1084B00079F08081803219F4442309F4492F8081B6
:1084C000803209F040E09F5F31968081882389F7F0
:1084D000442331F48081882311F4492F01C0462FB1
:1084E000262F3327E901C91BD109EC0FFD1F319657
:1084F000842F9927821B930B01971816190624F4D1
:10850000942F961B915001C090E091509F3F29F00D
:1085100081918D935F5F9150D8F71C925F5F852F9B
:108520009927DF91CF910895FC0190E081918823F4
:1085300031F09F5F8191882311F09F3FD1F7892F00
:1085400099270895DC01FB018081882329F081911E
:108550008D9380818823D9F71C9208950F931F93E0
:10856000CF93DF93082F162FFA0141E0C0E1D7E245
:10857000C901BE010E9424526115710581F06C9FF2
:10858000C0016D9F900D7C9F900D1124281B390B0D
:10859000862F805D8193440F01E015E00AC01530FD
:1085A00040F0002319F080E3819302C080E28193C0
:1085B0004F5FC8EED3E0C901BE010E94245261158D
:1085C000710581F06C9FC0016D9F900D7C9F900D97
:1085D0001124281B390B862F805D81934F5F01E0AA
:1085E00014E00AC0143040F0002319F080E38193B6
:1085F00002C080E281934F5FC4E6D0E0C901BE01B2
:108600000E9424526115710581F04F5F6C9FC0017B
:108610006D9F900D7C9F900D1124281B390B862F88
:10862000805D819301E013E00AC0133040F04F5F9A
:10863000002319F080E3819302C080E28193C90195
:108640006AE070E00E9424526115710591F04F5F5D
:10865000CB01880F991F880F991F880F991F860FCC
:10866000971F860F971F281B390B862F805D8193DC
:108670000AC0123040F04F5F002319F080E381936D
:1086800002C080E28193822F805D81931082842FCB
:108690009927DF91CF911F910F910895FC01262F0B
:1086A000862F82958F708A3038F06AE00E940452DB
:1086B000892F8F5B819309C0862F82958F706AE026
:1086C0000E940452892F805D8193822F8F708A309F
:1086D00038F06AE00E940452892F8F5B80830895EE
:1086E000822F8F706AE00E940452892F805D808300
:1086F0000895EF92FF920F931F937C018B01872FB8
:108700009927682FC7010E944E43C8019070682FB7
:10871000C7010E944E431F910F91FF90EF90089563
:10872000CF92DF92EF92FF920F931F936C017A0129
:108730008B01CB01AA27BB27BC01C6010E9479434C
:10874000D801C701A070B070BC01C6010E94794376
:108750001F910F91FF90EF90DF90CF9008951F939E
:10876000CF93DF93CDB7DEB769970FB6F894DEBF2E
:108770000FBECDBF10E0BE016F5F7F4F812F0E9403
:108780000E26212F3327C901880F991F880F991FA3
:10879000880F991F820F931FFC01EF52F44F8981BC
:1087A00085838A8186838B8187838C8180838D8179
:1087B00081838E8182838F81838388858483888D62
:1087C0008087F901EC54F34F10821F5F1F3098F23D
:1087D00069960FB6F894DEBF0FBECDBFDF91CF9183
:1087E0001F9108951F93CF93DF93CDB7DEB769979D
:1087F0000FB6F894DEBF0FBECDBF10E0A89519826A
:108800001A821B821C821D821E821F821886188E6D
:108810008FE0189FC001112489539A4FBC01CE01EB
:1088200009960E94C051BE016F5F7F4F812F0E9449
:10883000D6251F5F1F3010F369960FB6F894DEBF80
:108840000FBECDBFDF91CF911F910895CF93C0E0B0
:1088500086E0C89FC0011124FC01E65AF34FF09353
:10886000590CE093580C80819181009719F0019781
:1088700091838083E091580CF091590C828193810F
:10888000009719F0019793838283E091580CF0913F
:10889000590C84819581009719F001979583848301
:1088A0002C2F3327C901880F991F880F991F880F14
:1088B000991F820F931FFC01EF52F44F8081882390
:1088C00019F48181882321F08C2F8A5E0E942C4527
:1088D000CF5FCF3008F4BCCFCF9108959927873070
:1088E000910509F466C088309105ACF48430910597
:1088F00009F43EC08530910534F48230910511F1C0
:10890000039759F198C08530910509F43CC006974A
:1089100009F444C090C08A30910509F46BC08B30D3
:10892000910544F48830910509F44EC0099709F483
:1089300056C081C08B30910509F467C00C9709F4CB
:108940006FC079C080EC0E94B034882319F081E0B8
:1089500090E0089580E090E0089581EC0E94B034AA
:10896000882319F081E090E0089580E090E0089578
:1089700082EC0E94B034882319F081E090E00895E1
:1089800080E090E0089581ED0E94B034882319F0D2
:1089900081E090E0089580E090E0089584EC0E94EA
:1089A000B034882319F081E090E0089580E090E0F1
:1089B000089585EC0E94B034882319F081E090E09E
:1089C000089580E090E0089586EC0E94B0348823FA
:1089D00019F081E090E0089580E090E0089587EC40
:1089E0000E94B034882319F081E090E0089580E07F
:1089F00090E0089583EC0E94B034882319F081E060
:108A000090E0089580E090E0089582ED0E94B034F7
:108A1000882319F081E090E0089580E090E00895C7
:108A200083ED0E94B034882319F081E090E008952E
:108A300080E090E0089580E090E008959927FC019F
:108A4000ED54F34F80819927089524EB3CE0F90120
:108A5000E80FF11D60830895DF92EF92FF920F936C
:108A60001F93CF93DF93CDB7DEB721970FB6F8945E
:108A7000DEBF0FBECDBF1982863109F454C08731E5
:108A800019F481E089834FC0883119F482E0898329
:108A90004AC0893119F483E0898345C08A3119F4C9
:108AA00084E0898340C08B3119F485E089833BC021
:108AB0008C3119F486E0898336C08D3119F487E052
:108AC000898331C08E3119F488E089832CC08F31BD
:108AD00019F489E0898327C0803219F48AE08983F8
:108AE00022C0813219F48BE089831DC0823219F4CF
:108AF0008CE0898318C0833219F48DE0898313C018
:108B0000843219F48EE089830EC000E021E0AE01CA
:108B10004F5F5F4F6FE271E08EE591E00E94692147
:108B200080E090E0AFC6FF24EF2CDF2C298186E0A7
:108B3000289FC0011124865A934F9093590C80931B
:108B4000580C3327C901880F991F880F991F880F68
:108B5000991F820F931FFC01EF52F44F80818F3FCA
:108B600039F4EE24E394808580FF7DC1EF2C7BC136
:108B70008981282F332701ED1BE0C901880F991F38
:108B8000880F991F880F991F820F931FFC01E00F18
:108B9000F11FE0818E2F82508B3008F04CC08E2F59
:108BA0000E946E44482F8981282F3327C901880FDE
:108BB000991F880F991F880F991F820F931FFC011F
:108BC000E00FF11F808580FF02C081E04827442329
:108BD00069F0E091580CF091590C80819181892BBA
:108BE00019F4EE24E3943FC1EE243DC1A091580C4A
:108BF000B091590C8981282F3327C901880F991FFB
:108C0000880F991F880F991F820F931FFC01EF5245
:108C1000F44F958185E0989FC00111248D939C931A
:108C2000E091580CF091590C8081918101969183CB
:108C30008083EE2418C18981282F332701ED1BE0A2
:108C4000C901880F991F880F991F880F991F820FDC
:108C5000931FFC01E00FF11FE0818E2F8D508531B5
:108C600008F04CC08F5F0E94470A482F8981282F47
:108C70003327C901880F991F880F991F880F991FE3
:108C8000820F931FFC01E00FF11F808580FF02C05F
:108C900081E04827442369F0E091580CF091590C89
:108CA00080819181892B19F4EE24E394DCC0EE24B9
:108CB000DAC0A091580CB091590C8981282F332724
:108CC000C901880F991F880F991F880F991F820F5C
:108CD000931FFC01EF52F44F958185E0989FC001EE
:108CE00011248D939C93E091580CF091590C808144
:108CF0009181019691838083EE24B5C08981282FCC
:108D0000332701ED1BE0C901880F991F880F991FB8
:108D1000880F991F820F931FFC01E00FF11FE08164
:108D20008E2F8252823208F04CC08F5F0E94D51D78
:108D3000482F8981282F3327C901880F991F880F51
:108D4000991F880F991F820F931FFC01E00FF11FDD
:108D5000808580FF02C081E04827442369F0E091CC
:108D6000580CF091590C80819181892B19F4EE24D3
:108D7000E39479C0EE2477C0A091580CB091590CBF
:108D80008981282F3327C901880F991F880F991FC0
:108D9000880F991F820F931FFC01EF52F44F9581AA
:108DA00085E0989FC00111248D939C93E091580C0D
:108DB000F091590C80819181019691838083EE24FA
:108DC00052C08981282F3327C901880F991F880F26
:108DD000991F880F991F820F931F8C010F52144FF8
:108DE000F8019081892F84548F30E8F58F5F0E94BD
:108DF0001E45482FF801808580FF02C081E048278A
:108E0000442369F0E091580CF091590C80819181D4
:108E1000892B19F4EE24E39426C0EE2424C0A091FB
:108E2000580CB091590C8981282F3327C901880F1C
:108E3000991F880F991F880F991F820F931FFC019C
:108E4000EF52F44F958185E0989FC00111248D93D6
:108E50009C93E091580CF091590C8081918101967E
:108E600091838083EE248981282F3327C901880FBD
:108E7000991F880F991F880F991F820F931FFC015C
:108E8000EF52F44F81818F3F39F4FF24F3948085B2
:108E900081FF81C1FF247FC18981282F332701ED04
:108EA0001BE0C901880F991F880F991F880F991F10
:108EB000820F931FFC01E00FF11F9181892F8250D7
:108EC0008B3008F04DC0892F0E946E44482F898155
:108ED000282F3327C901880F991F880F991F880FE2
:108EE000991F820F931FFC01E00FF11F808581FF06
:108EF00002C081E04827442369F0E091580CF091CA
:108F0000590C82819381892B19F4FF24F39443C176
:108F1000FF2441C1A091580CB091590C8981282F90
:108F20003327C901880F991F880F991F880F991F30
:108F3000820F931FFC01EF52F44F968185E0989FBA
:108F4000C0011124FD0193838283E091580CF091BC
:108F5000590C82819381019693838283FF241BC1E4
:108F60008981282F332701ED1BE0C901880F991F44
:108F7000880F991F880F991F820F931FFC01E00F24
:108F8000F11F9181892F8D50853108F04DC08F5F81
:108F90000E94470A482F8981282F3327C901880F4B
:108FA000991F880F991F880F991F820F931FFC012B
:108FB000E00FF11F808581FF02C081E04827442334
:108FC00069F0E091580CF091590C82819381892BC2
:108FD00019F4FF24F394DFC0FF24DDC0A091580CE6
:108FE000B091590C8981282F3327C901880F991F07
:108FF000880F991F880F991F820F931FFC01EF5252
:10900000F44F968185E0989FC0011124FD01938360
:109010008283E091580CF091590C828193810196E2
:1090200093838283FF24B7C08981282F332701EDE2
:109030001BE0C901880F991F880F991F880F991F7E
:10904000820F931FFC01E00FF11F9181892F825243
:10905000823208F04DC08F5F0E94D51D482F898154
:10906000282F3327C901880F991F880F991F880F50
:10907000991F820F931FFC01E00FF11F808581FF74
:1090800002C081E04827442369F0E091580CF09138
:10909000590C82819381892B19F4FF24F3947BC0AE
:1090A000FF2479C0A091580CB091590C8981282FC8
:1090B0003327C901880F991F880F991F880F991F9F
:1090C000820F931FFC01EF52F44F968185E0989F29
:1090D000C0011124FD0193838283E091580CF0912B
:1090E000590C82819381019693838283FF2453C01C
:1090F0008981282F3327C901880F991F880F991F4D
:10910000880F991F820F931F8C010F52144FF80183
:109110009181892F84548F30F0F58F5F0E941E4516
:10912000482FF801808581FF02C081E04827442351
:1091300069F0E091580CF091590C82819381892B50
:1091400019F4FF24F39427C0FF2425C0A091580CE4
:10915000B091590C8981282F3327C901880F991F95
:10916000880F991F880F991F820F931FFC01EF52E0
:10917000F44F968185E0989FC0011124FD019383EF
:109180008283E091580CF091590C82819381019671
:1091900093838283FF248981282F3327C901880F75
:1091A000991F880F991F880F991F820F931FFC0129
:1091B000EF52F44F82818F3F39F4DD24D3948085C0
:1091C00082FF31C1DD242FC18981282F3327C901B6
:1091D000880F991F880F991F880F991F820F931F5F
:1091E000FC01EF52F44F9281892F82508B30C0F5F1
:1091F000892F0E946E44882369F0E091580CF09109
:10920000590C84819581892B19F4DD24D3940BC1E9
:10921000DD2409C1A091580CB091590C8981282FE7
:109220003327C901880F991F880F991F880F991F2D
:10923000820F931FFC01EF52F44F978185E0989FB6
:10924000C0011124FD0195838483E091580CF091B5
:10925000590C84819581019695838483DD24E3C034
:109260008981282F3327C901880F991F880F991FDB
:10927000880F991F820F931FFC01EF52F44F9281C8
:10928000892F8D508531C0F58F5F0E94470A882352
:1092900069F0E091580CF091590C84819581892BEB
:1092A00019F4DD24D394BFC0DD24BDC0A091580CB7
:1092B000B091590C8981282F3327C901880F991F34
:1092C000880F991F880F991F820F931FFC01EF527F
:1092D000F44F978185E0989FC0011124FD0195838B
:1092E0008483E091580CF091590C8481958101960A
:1092F00095838483DD2497C08981282F3327C90172
:10930000880F991F880F991F880F991F820F931F2D
:10931000FC01EF52F44F9281892F82528232C0F5C4
:109320008F5F0E94D51D882369F0E091580CF09161
:10933000590C84819581892B19F4DD24D39473C051
:10934000DD2471C0A091580CB091590C8981282F4F
:109350003327C901880F991F880F991F880F991FFC
:10936000820F931FFC01EF52F44F978185E0989F85
:10937000C0011124FD0195838483E091580CF09184
:10938000590C84819581019695838483DD244BC09B
:109390008981282F3327C901880F991F880F991FAA
:1093A000880F991F820F931FFC01EF52F44F928197
:1093B000892F84548F30B8F58F5F0E941E45882313
:1093C00069F0E091580CF091590C84819581892BBA
:1093D00019F4DD24D39427C0DD2425C0A091580CB6
:1093E000B091590C8981282F3327C901880F991F03
:1093F000880F991F880F991F820F931FFC01EF524E
:10940000F44F978185E0989FC0011124FD01958359
:109410008483E091580CF091590C848195810196D8
:1094200095838483DD244981842F99279C01220F11
:10943000331F220F331F220F331F280F391FF9014B
:10944000EF52F44F8081882309F45AC18181882327
:1094500009F456C18281882309F452C1838188238B
:1094600009F077C0EE20C9F1FF20B9F1848188238B
:1094700061F46D2D842F0E942545DD2019F081E0D7
:1094800090E000C280E090E0FDC18981282F332761
:10949000C901880F991F880F991F880F991F820F84
:1094A000931FFC01EF52F44F8481823079F460E025
:1094B000ED1409F461E089810E942545ED1419F449
:1094C00081E090E0DFC180E090E0DCC161E0898173
:1094D0000E94254581E090E0D5C14981242F3327A2
:1094E000C901880F991F880F991F880F991F820F34
:1094F000931FFC01EF52F44F8481823049F4DD2048
:1095000039F461E0842F0E94254581E090E0BAC1E2
:109510004981842F99279C01220F331F220F331F6B
:10952000220F331F280F391FF901EF52F44F6481C6
:10953000613041F4DD2031F0842F0E94254581E027
:1095400090E0A0C160E089810E94254580E090E024
:1095500099C14981842F99279C01220F331F220F23
:10956000331F220F331F280F391FF901EF52F44F19
:109570008381823009F040C0EF14B9F584818823DB
:1095800061F46D2D842F0E942545DD2019F081E0C6
:1095900090E078C180E090E075C18981282F332761
:1095A000C901880F991F880F991F880F991F820F73
:1095B000931FFC01EF52F44F8481823079F460E014
:1095C000ED1409F461E089810E942545ED1419F438
:1095D00081E090E057C180E090E054C161E0898172
:1095E0000E94254581E090E04DC160E089810E94A4
:1095F000254580E090E046C1EE2019F4FF2009F4F3
:1096000043C04981242F3327C901880F991F880F30
:10961000991F880F991F820F931FFC01EF52F44F7F
:109620008481882361F46D2D842F0E942545DD20DF
:1096300019F081E090E026C180E090E023C14981EB
:10964000242F3327C901880F991F880F991F880F6E
:10965000991F820F931FFC01EF52F44F84818230D7
:1096600061F46D2D842F0E942545DD2019F081E0E5
:1096700090E008C180E090E005C161E089810E942E
:10968000254581E090E0FEC04981842F99279C0107
:10969000220F331F220F331F220F331F280F391FB2
:1096A000F901EF52F44F6481613041F4DD2009F19A
:1096B000842F0E94254581E090E0E4C04981242F59
:1096C0003327C901880F991F880F991F880F991F89
:1096D000820F931FFC01EF52F44F8481823049F4D2
:1096E000DD2039F461E0842F0E94254581E090E07F
:1096F000C9C060E089810E94254580E090E0C2C039
:109700004981842F99279C01220F331F220F331F79
:10971000220F331F280F391FF901EF52F44F8081B8
:10972000882309F44DC08181882309F449C08381CD
:10973000882391F4EE2049F0FF2039F061E0842F76
:109740000E94254581E090E09DC060E089810E94F3
:10975000254580E090E096C04981242F3327C90138
:10976000880F991F880F991F880F991F820F931FC9
:10977000FC01EF52F44F8381823081F4EF1439F40D
:1097800061E0842F0E94254581E090E07BC060E08D
:1097900089810E94254580E090E074C0EE2011F49C
:1097A000FF2039F061E089810E94254581E090E049
:1097B00069C060E089810E94254580E090E062C038
:1097C0004981842F99279C01220F331F220F331FB9
:1097D000220F331F280F391FF901EF52F44F8181F7
:1097E000882309F44DC08281882309F449C084810B
:1097F000882391F4EE2049F0FF2039F061E0842FB6
:109800000E94254581E090E03DC060E089810E9492
:10981000254580E090E036C04981242F3327C901D7
:10982000880F991F880F991F880F991F820F931F08
:10983000FC01EF52F44F8481823081F4EF1439F44B
:1098400061E0842F0E94254581E090E01BC060E02C
:1098500089810E94254580E090E014C0EE2011F43B
:10986000FF2039F061E089810E94254581E090E088
:1098700009C060E089810E94254580E090E002C037
:1098800080E090E021960FB6F894DEBF0FBECDBF0A
:10989000DF91CF911F910F91FF90EF90DF9008958E
:1098A000CF93DF93CDB7DEB721970FB6F894DEBF25
:1098B0000FBECDBF282F04B603FE28C0FE0131968F
:1098C000ACEBB0E081E090E031E08030930719F438
:1098D0000E94B35203C0182E0E94B3528981843172
:1098E00090F48F5F8983FE013196ACEBB0E081E0AC
:1098F00090E031E08030930719F40E94C45203C015
:10990000182E0E94C45284B7877F84BF8091600064
:10991000886180936000209360008091600088607F
:109920008093600021960FB6F894DEBF0FBECDBFC6
:10993000DF91CF910895EF92FF920F931F937B01D8
:109940008C0120E030E040E05FE40E94FF4E88237D
:109950009CF020E030E040E05FECC801B7010E94DD
:10996000E94DDC01CB01BC01CD010E94994F605053
:1099700070408040904804C0C801B7010E94994FD0
:109980001F910F91FF90EF900895A0E0B0E0EBECF5
:10999000FCE40C9474528C017B015A01DC018C9123
:1099A000823058F0FB019081923010F4A7010BC176
:1099B000843029F4943009F4A6C0A80104C194307D
:1099C000A9F3923009F4A9C0823081F3F801C28072
:1099D000D380FB0162817381F80124813581468146
:1099E0005781F7016480758086809780C601861B49
:1099F000970B97FDD8C080970CF46CC06C157D0553
:109A00000CF0ADC0662477244301F8016181F701B1
:109A10008181681709F499C0662309F491C0621A1C
:109A2000730A840A950AA401930157FDC0C0F50189
:109A30001182B60119012A0179018A0139014A010D
:109A400008946108710881089108FFEF6F16FFEF15
:109A50007F06FFEF8F06FFE39F06F0F4A801970152
:109A6000220F331F441F551F19012A01B6016150EF
:109A700070406B0179018A0139014A01089461083B
:109A80007108810891088FEF68168FEF78068FEFC5
:109A900088068FE3980610F383E0D5018C9357FC7A
:109AA00064C0F501248335834683578373836283BF
:109AB000A50189C06F5F7F4FD401C3018170907091
:109AC000A070B0709694879477946794682A792AE6
:109AD0008A2A9B2A6C157D056CF311C00894C11C61
:109AE000D11CDA01C90181709070A070B0705695D8
:109AF000479537952795282B392B4A2B5B2BC61674
:109B0000D70664F382CFF8019181FB018181981718
:109B100009F453CF41E751E056C0823009F04DCFF0
:109B200088E0DA01F80101900D928A95E1F7F801D9
:109B30008181FB0191818923FA018183A50143C0C1
:109B4000261937094809590970CFF5016183B60113
:109B5000260D371D481D591D19012A019DCF6B0186
:109B600020E030E040E050E050CFD201C101B69596
:109B7000A7959795879521E030E040E050E02222BC
:109B8000332244225522282A392A4A2A5B2AF501FF
:109B900024823582468257820894C11CD11CD3820C
:109BA000C282A50110C0909581959F4F24CF81E07E
:109BB000F5018183B60150954095309521953F4F31
:109BC0004F4F5F4F37CFCA01E2E1CDB7DEB70C94FC
:109BD0009052A0E2B0E0EFEEFDE40C948252DC0182
:109BE000CB01898F9A8FAB8FBC8F2D8F3E8F4F8F7C
:109BF00058A3BE016F5F7F4FCE0149960E94D3509C
:109C00008E01075F1F4FB801CE014D960E94D350C1
:109C1000AE014F5E5F4FB801CE0101960E94C54C68
:109C20000E94EB4FDC01CB01BC01CD01E4E0A0962A
:109C30000C949E52A0E2B0E0E0E2FEE40C9482526A
:109C4000DC01CB01898F9A8FAB8FBC8F2D8F3E8F1C
:109C50004F8F58A3BE016F5F7F4FCE0149960E9480
:109C6000D3508E01075F1F4FB801CE014D960E9461
:109C7000D3508A8591E089278A87AE014F5E5F4F76
:109C8000B801CE0101960E94C54C0E94EB4FDC0149
:109C9000CB01BC01CD01E4E0A0960C949E52A8E15A
:109CA000B0E0E5E5FEE40C947C52DC01CB01898B4D
:109CB0009A8BAB8BBC8B2D8B3E8B4F8B588FBE0101
:109CC0006F5F7F4FCE0141960E94D3508E01075F98
:109CD0001F4FB801CE0145960E94D350FE01319628
:109CE0002981223008F45FC03985323010F4B80180
:109CF0007BC081819A8589278183243009F455C0EE
:109D0000223009F452C0343009F454C0323009F41E
:109D100058C06B817C818B859C85681B790B2D815C
:109D20003E814F815885ED84FE840F8518892E155C
:109D30003F054007510730F4220F331F441F551FC2
:109D4000615070407C836B8380E090E0A0E0B0E4E1
:109D5000AA24BB2465012E153F054007510740F09A
:109D6000A82AB92ACA2ADB2A2E193F09400B510B0F
:109D7000B695A79597958795220F331F441F551FBA
:109D80000097A105B10539F7D601C5018F7790700D
:109D9000A070B07080349105A105B105A9F0A4822E
:109DA000B582C682D782BF011FC02317E1F761E7E2
:109DB00071E01AC01D821E821F8218861C821B82BF
:109DC000F2CF84E08983EFCFA7FC05C021153105D0
:109DD0004105510521F380E490E0A0E0B0E0A80E39
:109DE000B91ECA1EDB1EDBCFCB010E94EB4FDC018C
:109DF000CB01BC01CD01EAE068960C949852A8E131
:109E0000B0E0E5E0FFE40C948252DC01CB01898BE9
:109E10009A8BAB8BBC8B2D8B3E8B4F8B588FBE019F
:109E20006F5F7F4FCE0141960E94D3508E01075F36
:109E30001F4FB801CE0145960E94D35089818230D0
:109E400018F08985823018F42FEF3FEF09C0B80170
:109E5000CE0101960E944D51282F332727FD3095C2
:109E6000C901E4E068960C949E52A8E0B0E0EBE3F0
:109E7000FFE40C9480529B01AC017B018C01EE2429
:109E800017FDE394FF2400271127EA8221153105ED
:109E90004105510539F482E08983CE0101960E9483
:109EA000EB4F43C083E089836EE170E0CB01EE208D
:109EB00031F579018A01A80197012030E0E03E07E1
:109EC000E0E04E07E0E45E0798F479018A01EE0CC9
:109ED000FF1C001F111F0197BC01A8019701E0E0C2
:109EE000EE16E0E0FE06E0E00E07E0E41E0768F391
:109EF000ED82FE820F8318877C836B83CECF203068
:109F0000E0E03E07E0E04E07E0E85E0741F0EE24C7
:109F1000FF248701E21AF30A040B150BCCCF7C83D4
:109F20006B8360E070E080E09FECE6E028960C94A4
:109F30009C52ACE0B0E0EFE9FFE40C948452DC0109
:109F4000CB0189879A87AB87BC87BE016F5F7F4F44
:109F5000CE0109960E94D3508981823011F082305F
:109F600028F460E070E080E090E031C0843039F0A7
:109F70002B813C8137FDF5CF2F3131056CF08A8183
:109F8000882329F060E070E080E090E820C06FEF67
:109F90007FEF8FEF9FE71BC08EE190E0821B930B5A
:109FA0002D813E814F81588504C056954795379540
:109FB00027958A95D2F78A81882339F05095409564
:109FC000309521953F4F4F4F5F4FCA01B901E2E0F5
:109FD0002C960C94A052A0E0B0E0E1EFFFE40C94CA
:109FE0007A52882499245401DC01FC0124813581B2
:109FF000468157818181082F112760E070E08C91A4
:10A00000823020F46FEF70E04061A4C0843009F426
:10A0100064C0823009F463C0211531054105510542
:10A0200009F498C0FD0182819381FFEF82389F0778
:10A030000CF050C0A2E8EA2EAFEFFA2EE81AF90AA7
:10A040008AE1E816F1040CF06BC06B0181E090E04E
:10A05000A0E0B0E00E2C04C0880F991FAA1FBB1F00
:10A060000A94D2F70197A109B10982239323A4236B
:10A07000B5230097A105B10519F0F1E0CF2ED12C41
:10A0800004C05695479537952795EA94D2F7C601AF
:10A09000AA2797FDA095BA2F282B392B4A2B5B2B8B
:10A0A000DA01C9018F779070A070B070803491058B
:10A0B000A105B105D1F1215C3F4F4F4F5F4F2030DB
:10A0C000E0E03E07E0E04E07E0E45E0708F161E013
:10A0D00070E01EC0803891053CF06FEF70E020E02A
:10A0E00030E040E050E036C0BC0161587F4FDA01FB
:10A0F000C9018F779070A070B07080349105A10570
:10A10000B105D1F0215C3F4F4F4F5F4F57FD1BC052
:10A1100097E056954795379527959A95D1F71AC0A8
:10A1200020E030E040E050E0BBCF27FFC8CF205C0C
:10A130003F4F4F4F5F4FC3CF27FFE8CF205C3F4FCC
:10A140004F4F5F4FE3CF56954795379527956F5FF4
:10A150007F4FDECF822E932E942F9F778A2D80788B
:10A16000A82EA92A962F9795992797958A2D8F77AC
:10A17000A82EA92A76956795962F9F778B2D8078A4
:10A18000B82EB92A902F9795992797958B2D8F7771
:10A19000B82EB92AD501C401BC01CD01ECE0CDB780
:10A1A000DEB70C949652CF93DF93FC01DB01408124
:10A1B00051812281622F6F7770E0221F2227221F98
:10A1C0009381892F880F822B282F3327991F992756
:10A1D000991FED0199832115310541F44115510570
:10A1E00061057105E1F482E08C9354C02F3F310585
:10A1F00009F441C02F573040FD013383228383E0AF
:10A200008C9387E0440F551F661F771F8A95D1F7FF
:10A210007064ED014C835D836E837F833BC022E8D5
:10A220003FEFF901C7E0440F551F661F771FCA951E
:10A23000D1F783E08C93403080E0580780E06807D6
:10A2400080E4780778F4440F551F661F771F21506C
:10A250003040F9014030C0E05C07C0E06C07C0E46A
:10A260007C0788F3ED01FB83EA83FD01448355837A
:10A27000668377830FC0411551056105710519F497
:10A2800084E08C9307C064FF03C081E08C93C1CF4E
:10A290001C92BFCFDF91CF9108950F931F93CF935F
:10A2A000DF93FC01DB018081823018F09C919230B9
:10A2B00018F461E070E05EC08430C1F0843001F1D8
:10A2C000943009F447C0823009F44BC0823009F45D
:10A2D0004EC09230A9F04181ED0189814817B9F053
:10A2E000442389F08FEF9FEFBC0144C0943031F7D5
:10A2F000EB018981682F77278181681B71093AC03A
:10A300008181882379F781E090E0BC0133C022810C
:10A310003381ED018A819B81821793070CF3281703
:10A3200039079CF00481158126813781FD01648104
:10A33000758186819781601771078207930780F284
:10A34000061717072807390778F4442359F281E0E4
:10A3500090E0DBCFFD018181882321F281E090E054
:10A36000D4CF923009F0B2CF60E070E003C0ED01CD
:10A370008981F2CFCB01DF91CF911F910F91089589
:10A38000FB01DC0105900D920020E1F70895FB012F
:10A39000DC0140FF05C002C001900D9201900D92BA
:10A3A00042505040C8F70895DC0140FF03C001C08F
:10A3B0006D936D9342505040D8F70895FB01DC0136
:10A3C00001900D920020E1F70895629FD001739FE4
:10A3D000F001829FE00DF11D649FE00DF11D929F41
:10A3E000F00D839FF00D749FF00D659FF00D992780
:10A3F000729FB00DE11DF91F639FB00DE11DF91FA4
:10A40000BD01CF0111240895991B79E004C0991F63
:10A41000961708F0961B881F7A95C9F780950895BE
:10A42000AA1BBB1B51E107C0AA1FBB1FA617B7077A
:10A4300010F0A61BB70B881F991F5A95A9F7809596
:10A440009095BC01CD01089597FB092E07260AD0EF
:10A4500077FD04D0E5DF06D000201AF470956195F1
:10A460007F4F0895F6F7909581959F4F0895A1E24B
:10A470001A2EAA1BBB1BFD010DC0AA1FBB1FEE1F7E
:10A48000FF1FA217B307E407F50720F0A21BB30BC9
:10A49000E40BF50B661F771F881F991F1A9469F745
:10A4A00060957095809590959B01AC01BD01CF01A1
:10A4B000089597FB092E05260ED057FD04D0D7DF4F
:10A4C0000AD0001C38F450954095309521953F4FA7
:10A4D0004F4F5F4F0895F6F7909580957095619571
:10A4E0007F4F8F4F9F4F08952F923F924F925F92D1
:10A4F0006F927F928F929F92AF92BF92CF92DF9294
:10A50000EF92FF920F931F93CF93DF93CDB7DEB7F8
:10A51000CA1BDB0B0FB6F894DEBF0FBECDBF09948C
:10A520002A88398848885F846E847D848C849B84E3
:10A53000AA84B984C884DF80EE80FD800C811B81F1
:10A54000AA81B981CE0FD11D0FB6F894DEBF0FBE20
:10A55000CDBFED010895F999FECFB2BDA1BDF89A26
:10A56000119600B40895F7DF01921A94E1F7089567
:10A57000F999FECFB2BDA1BD00BC11960FB6F894FB
:10A58000FA9AF99A0FBE08950190F2DF1A94E1F752
:02A5900008952C
:10A5920001012E2E2F63616E5F696E7075742E63DA
:10A5A200006E2E2E2F6368616E6E656C732E6300D3
:10A5B200455231002E2E2F656570726F6D63686192
:10A5C2006E6E656C732E630050434D300045523100
:10A5D200004C4F4730340050434D2076657220378F
:10A5E2002E3436004F4252203834343009002E2E99
:10A5F2002F7669727475656C5F696E7075742E63FF
:0AA60200000000000000000000004E
:00000001FF
